:020000040000FA
:060000000200B20222D44E
:03002300021F19A0
:03002B000222E8C6
:10003B0002218153D9BF79012200000080FB1200FD
:10004B003EB900030200ACE479217842B80002808B
:10005B0004F709D8FCE49001A1788779088002F0B5
:10006B00A3D8FCD9FA78129000C17A01BA000280A9
:10007B0007E493A3F608DAF9900927AA82AB8390D9
:10008B0000C2789B79038015E493A3AC82AD838A7D
:10009B00828B83F0A3AA82AB838C828D83D8E9D920
:1000AB00E712364712004475D0007581BF7510A159
:1000BB0075110102004940506C65617365207072C7
:1000CB0065737320616E79206B657920746F206383
:1000DB006F6E74696E75652E2E2E203F007C203658
:1000EB0034207B207C203530306E732F64207C20B5
:1000FB0035302E30562F64207C2035302E30562F45
:10010B0064207C3F007C2053796E63207C20496EF9
:10011B0074207C205A20434841207C205A2043489D
:10012B0042207C204143204143207C3F0035302E30
:10013B0030562F643F0041433F00204143203F0096
:10014B00204443203F00436F6C6F72204348204193
:10015B003F00436F6C6F7220434820423F00426167
:10016B00636B20436F6C6F723F004175746F20435C
:10017B006F7272656374696F6E205A65726F3F00A0
:10018B004578697420616E6420536176653F004544
:10019B0078697420776974686F757420536176651C
:1001AB003F004368616E6E656C20413F0052616E8B
:1001BB0067653A3F004F4B203F006661696C757273
:1001CB00653A3F004368616E6E656C20423F005399
:1001DB0075636365737366756C6C7920626F746895
:1001EB00206368616E6E656C733F00537563636566
:1001FB00737366756C6C79206F6E6C7920636861B4
:10020B006E6E656C20413F00537563636573736657
:10021B00756C6C79206F6E6C79206368616E6E659E
:10022B006C20423F004661696C7320666F722062DE
:10023B006F7468206368616E6E656C733F005072FB
:10024B0065737320616E79206B657920746F206301
:10025B006F6E74696E75653F0050432052554E208A
:10026B004D4F44453F0044433F00496E743F0025CA
:10027B0068640053796E633F003634207B3F005532
:10028B0000070700025980203634207B203F0000F6
:10029B0000203530306E732F64203F2035302E30E8
:1002AB00562F64203F2035302E30562F64203F20B0
:1002BB0053796E63203F00000020496E74203F008D
:1002CB00000000205A20434841203F0000205A20C4
:1002DB00434842203F000020464654203F00000088
:1002EB00000000000000000000000001E52FE6FF09
:1002FB0000F8010101000000002C010000010000CA
:10030B0000409C00003031323334353637383941B8
:10031B00424344454600286E756C6C20706F696EC5
:10032B0074657229003F3F3F000000807F00008012
:10033B003FF9021550B743BA510000204100E7DBEB
:10034B002E0000A04010000000080000000A000072
:10035B0000C3E09608A3E09608A3E09608A3E096F6
:10036B00A2D265D03322C008C3E096F50808A3E0FB
:10037B0096420808A3E096420808A3E0964208A21A
:10038B00D265D033E5087001D3D00822080808E6FF
:10039B0030E711120C3B1203AF080808C64480C6A5
:1003AB0018181822181818E9799EC608CAC608CB5F
:1003BB00C608CCC6C370207996CACBCC7019798E7F
:1003CB00CBCC70137986CC700EF9802ACA33CACB8A
:1003DB0033CBCC33CC331930E7F2CCCBCA335014FC
:1003EB007004EA30E00DE4CA3ACACB3BCBCC3CCC30
:1003FB00500209C3E913C6CC182313C6CB18C6CABF
:10040B0018C6F92212044F20F01430E72B74FFFCAE
:10041B00FBFA747F8022E4FCFBFA7480801AB480B0
:10042B0008BC00F2BB00EF800F50EBF9E4C39AFA63
:10043B00E49BFBE49CFCE499C6CC18C6CB18C6CA5B
:10044B0018C6F922E4C9C608CAC608CBC6D33303FB
:10045B0008CCC63392F0C3947F402E94184019C930
:10046B00B90704CACBCC225025C309CA33CACB3334
:10047B00CBCC33CC33D9F422F4600DC9CCC313CB22
:10048B0013CBCA13CAD9F6CC22E4FCFBFA2214FC18
:10049B00FBFA22E6C33318461846184622E7C33345
:1004AB0019471947194722181818E6084608700A01
:1004BB00E608C3337005E633F4220822191919E74D
:1004CB00094709700AE709C3337005E733F42209BA
:1004DB0022E6084608C3134608336002E633F422CB
:1004EB00E7094709C3134709336002E733F42212C4
:1004FB0004DC60251204EB602012049E70030204DE
:10050B00A8080808E76670101819E766700A18192A
:10051B00E76670041819E76622F4221204DC601CEB
:10052B001204EB601712049E70071204A87001D31B
:10053B0022C0D01204A87006D0D0B322C32233D06D
:10054B00D0501430E0F6C3E7960809E7960809E7A0
:10055B00960809E796B32220E0D5E6970809E697B7
:10056B000809E6970809E697B3221204DC601B1210
:10057B0004EB601612049E70071204A8600CB322E1
:10058B00C0D01204A87005D0D022C32233D0D050D3
:10059B001330E0EBC3E7960809E7960809E79608DE
:1005AB0009E7962220E0E4E6970809E6970809E6B2
:1005BB00970809E69722001204DC604F1204EB60E7
:1005CB0012E7548066F61204B270111204A8703B45
:1005DB00090909F4F618F618F618F6221204C77072
:1005EB001512049E08080860EAE6447FF618768028
:1005FB0018E4F618F62212049E60161204A8701264
:10060B00E4F608F608F608E65480F6090909181806
:10061B001822EAC0E0EBC0E0ECC0E0EDC0E0E687FA
:10062B00F0A4FBACF008E687F0A42CFCE435F0FA60
:10063B001809E687F0A42C4B60027401CA35F0FC54
:10064B00E433FB09E687F0D2F7A42CCB35F0FC1989
:10065B0008E687F0A42BCC35F0FBE433FD0819E654
:10066B0087F0D2E7A42C4ACB35F0CD3400FC09E659
:10067B0087F0D2E7A42DCC35F0FDE433FA0918E668
:10068B0087F0D2F7A42CCD35F0CA3400FC08E687EE
:10069B00F0D2E7D2F7A42ACC35F07A7E20E70B0A0A
:1006AB00CB33CBCD33CDCC33CC33CB3350147004D5
:1006BB00ED30E00ED2F1E4CD3DCDCC3CCC3B500542
:1006CB00DA05C2F1EB547FC63308E63392F0FBE751
:1006DB003309E733C39A502D2B70190C0D4C4D7009
:1006EB00151806E608C333700D20F10AA2F013F6B5
:1006FB00E418800B4024E4F630F002768018F618EC
:10070B00F618F68024D33B14501074FFA2F013F6A6
:10071B00187680E418F618F6800FA2F013F618E698
:10072B003303F618ECF618EDF6D0E0FDD0E0FCD074
:10073B00E0FBD0E0FA221204EB60461204DC603DD1
:10074B00E9687008F618F618F618F622748067F741
:10075B00120775090909748067F7221204DC601D02
:10076B001204EB7005191919801A1204B2701F12BA
:10077B0004C7C37003E66733191919400718181813
:10078B002208080874FFF618F618F618F622120459
:10079B00C760171204A8702192F012049E701950B2
:1007AB001720F014080808090909E7F61819E7F6E5
:1007BB001819E7F61819E7F62212049E60E6E869A5
:1007CB00701F0808E62480F608E436F618547FB448
:1007DB007F0CE654806007F6E418F618F62218181A
:1007EB0022E9C6CC08C6CD08C6CE08C6CFC0E0E805
:1007FB00C0E0EAC0E0EBC0E009E9F809E7FA09E775
:10080B00FBE6F918E6F8C3EC98ED99EE9AEBC2E724
:10081B00F5F0EFC2E795F0500E600CEBCFFBEACE94
:10082B00FAE9CDF9E8CCF8EAA2E7D2E7FAEB33FB29
:10083B0013F5F0EEA2E7D2E7FEEF33FFC5F013A2FC
:10084B00E730E601B313C5F0C3C0E0C0F07F00C3CF
:10085B009BFB605B9418600C401AD0E023F9D0E04E
:10086B00F80209448AF0E9486003D2F0E4AFF0FAE9
:10087B00F9F8803BEB30E40D89F0EA6003D2F0E449
:10088B00AFF0F9CAF8EB30E30D88F0EF6002D2F06D
:10089B00AFF0E4CAC9F8EB54076014FBC3EA13FAD0
:1008AB00E913F9E813F8EF135002D2E0FFDBEDD0B8
:1008BB00E0C0E030E739C3E49FFFF5F0EC98FC4271
:1008CB00F0ED99FD42F0EE9AFE42F0D0E0F9D0E067
:1008DB00F8E5F0607AE923F9EE20E742D802806769
:1008EB00C3EF33FFEC33FCED33FDEE33FE80EAEC6C
:1008FB0028FCED39FDEE3AFED0E023F9D0E0F840CC
:10090B0002801BC3EE13FEED13FDEC13FCEF135033
:10091B0002D2E0FF08B800067F7F74FF802EEF3312
:10092B0050178CF020F00260100CBC000C0DBD00B9
:10093B00080EBE000408E860DFE933E813FFEE237E
:10094B0013FE4F4D4C8008E95480FFE4FEFDFCEE96
:10095B0033EF33F47004FCFD7E80D0E0FBD0E0FA83
:10096B00D0E0F8D0E0CFC618CEC618CDC618CCC68E
:10097B00F9221204DC7004181818221204EB700D03
:10098B0074FFF61819F61819F61819F622E75480A1
:10099B0066F612049E700F1204A870F014F608F697
:1009AB0008F608F680D11204A8700CF608F6087643
:1009BB008008E6447F80EC1204CA700C1204B56008
:1009CB00BFE65480F6E480BB1204B5700519191903
:1009DB0080A5E869700C763F18768018F618F6E853
:1009EB00F922E6CDC0E018ECC0E0E633CD33CDD331
:1009FB0013F6E719FCE7191933CC33C3947F400E78
:100A0B00CD9D502408E65480F6E418F6800FF404CC
:100A1B003D14501408E6447FF6187680E418F61857
:100A2B00F6D0E0FCD0E0FD22CCD313CCFD18E4C60D
:100A3B00CBC0E018E4C6CAC0E00808ED08C633E630
:100A4B0013F618E433C675F003C3CA97CA09CB97DC
:100A5B00CB199C40047D08802EBD0003020B26168B
:100A6B00B6FF050606081618C3CA33CACB33CB33F9
:100A7B00CA27CA09CB37CB193CC37D08803E187DEA
:100A8B000820E75CC633C6CA33CACB33CB33DDF1A0
:100A9B00D5F0EB30E77BCA97CA09CB974ACB199CA9
:100AAB00406F4B7025E620E0218066187D08C3CA95
:100ABB0097CA09CB97CB199CD3C633C6CA33CACBBB
:100ACB0033CB3350C9DDE7D5F0E1D3E4C636C608E6
:100ADB00C636C608C636C608C636C61818188031BC
:100AEB00C3CA97CA09CB97CB199CB34097C633C6D9
:100AFB00CA33CACB33CB33DD34D5F02EC6A2E0C616
:100B0B0040C8CA27CA09CB37194A70BECB3CB48040
:100B1B00B90808E63308E633601F181818D0E0FA56
:100B2B00D0E0FBD0E0FCD0E0FD22187D08CA27CA3C
:100B3B0009CB37CB193CD3808013F618E4B67F1161
:100B4B00F618B6FF0EF618C60470D2080876808029
:100B5B00CAF618F618F680C5E4CFC0E0E4CEC0E0C4
:100B6B00E4CDC0E0E4CCC0E075F020C3E633F6087A
:100B7B00E633F608E633F608E633F6181818EC33C6
:100B8B00FCED33FDEE33FEEF33FFC3EC9709ED972E
:100B9B0009EE9709EF97191919400FFFEC97FC090C
:100BAB00ED97FD09EE97FE191906D5F0BEECF70986
:100BBB00EDF709EEF709EFF7191919D0E0FCD0E0C2
:100BCB00FDD0E0FED0E0FF22120C3E181818120BDD
:100BDB0063120C2A19191922120C2A19191908084F
:100BEB0008E618181820E7E0120B63120C3E1818D1
:100BFB001822090909E719191920E7DC080808E682
:100C0B0018181820E703020B63120C3E1818181261
:100C1B000B63120C3E181818120C2A19191922E41E
:100C2B00C397F709E497F709E497F709E497F722D5
:100C3B00181818E4C396F608E496F608E496F60836
:100C4B00E496F622E627F60809E637F60809E637B2
:100C5B00F60809E637F622E026F008A3E036F0089E
:100C6B00A3E036F008A3E036F022E0F608A3E0F6A6
:100C7B0008A3E0F608A3E0F622E6F008A3E6F008E6
:100C8B00A3E6F008A3E6F022E0FAA3E0FBA3E0FC66
:100C9B00A3E0FD22EAF0A3EBF0A3ECF0A3EDF0222E
:100CAB00CAC0E0E6F0A308DAFAD0E0FA22CAC0E044
:100CBB00E0A3C582CCC582C583CDC583F0A3C58215
:100CCB00CCC582C583CDC583DAE6D0E0CA22C3E4A6
:100CDB0098F8E499F9120D1A8026C3E49AFAE49B6A
:100CEB00FBE920E7E9120D1AE498F8E499F922C31D
:100CFB00E498F8E499F9120D1AE498F8E499F9C319
:100D0B00E49AFAE49BFB22EB20E7CFE920E7E0B97A
:100D1B000010BB0008E88AF084F8AAF022E4FBC8B4
:100D2B00FA22EB70227B10C833C8C933C933500782
:100D3B00C39AC3DBF280069A50012ADBEAC833F46C
:100D4B00C8C933F4C9FA2275F008E4C833C8C933EB
:100D5B00C933C99AC99B5004C92AC93BD5F0ECFBCE
:100D6B00C833F4C8E4C9FA22600D08C6A2E713C65B
:100D7B0018C613C6D5E0F322700422600D18C6C343
:100D8B0033C608C633C6D5E0F41822251010AF08B9
:100D9B00F510400215118008F51040021511D2AF65
:100DAB0022C0D0251010AF08F51050020511800895
:100DBB00F51050020511D2AFD0D0222510F58210BC
:100DCB00AF08F510400215118008F51040021511FF
:100DDB00D2AF851183222510F582E43511F58322DC
:100DEB00E473C0E0E8C0E0E58124FCF8E6A2E7D0BC
:100DFB00E0F8D0E0222510C582C0E0E51134FFC534
:100E0B0083C0E0E510C3958224F910AF08858311E8
:100E1B008582108008858311858210D2AFCEF0A316
:100E2B00E520F0A37808E608F0A3DEFAEFF0A3E5DF
:100E3B008124FBF8E608F0A3E608F0A30808E6080F
:100E4B00F0A3E608F0A315811581D0E0FED0E0F801
:100E5B0015811581E8C0E0EEC0E022851183851075
:100E6B0082E0A3FEE0A3F5207808E0A3F608DFFA02
:100E7B00E0A3FFE0A3C0E0E0A3C0E0E0A3C0E0E09C
:100E8B00A3C0E010AF08858210858311800885828E
:100E9B0010858311D2AFD083D0822274028002746A
:100EAB0001C0E0F404120DC6D0E0120CAB227402A8
:100EBB008000CCC0E0EDC0E0E510C39CCCAD115080
:100ECB00011D10AF068C108D1180068C108D11D268
:100EDB00AF120CB8D0E0FDD0E0FC22D083D082E979
:100EEB00C0E0E493A3C386F0C5F095F0F908E49352
:100EFB00A386F0C5F095F0700BE493A3C39940055E
:100F0B00E9048002A3E475F002A42582F582E5F0E2
:100F1B003583F583D0E0F9E493A3C0E0E493C0E01C
:100F2B002275B9807414001470FC43B9C0E5B9A2E2
:100F3B00E550FA75A90275B28322C082C083120FE5
:100F4B002C75A40D75A5E775A70175D40F75D5077D
:100F5B0075DF0175E10575E242D28875E401D2A80F
:100F6B00C2AA75C80475CA0175CB01C2AD759810BC
:100F7B00538EF4438E08858D8B758DF353890F43F8
:100F8B008920D28E900B5B7401F0D2BCD2ACD28C88
:100F9B00438922438E0C758CB075C18043E6017575
:100FAB00D80053D9BF75D90275DA4275DB4275FC8F
:100FBB000775EA07D2DEC283D282D280C292D29167
:100FCB00D290D2B0C296D296D2AF021F14D296D282
:100FDB0082D29275A6FFD291C291D291D283C29244
:100FEB0075A083C280D280D29275A002C280D280BB
:100FFB00C283D283C29275A085C280D280D29275F1
:10100B00A003C280D280C283D283C29275A08CC24D
:10101B0080D280D29275A093C280D280C283D283B9
:10102B00C29275A091C280D280D29275A001C2806B
:10103B00D280C283D283C29275A083C280D280D267
:10104B009275A000C280D280C283D283C29275A057
:10105B003EC280D280D29275A0B0C280D280C283B1
:10106B00D283C29275A03FC280D280D29275A00368
:10107B00C280D280C283D283C29275A040C280D27A
:10108B0080D29275A010C280D280C283D283C292CA
:10109B0075A041C280D280D29275A056C280D280F8
:1010AB00C283D283C29275A042C280D280D2927583
:1010BB00A013C280D280C283D283C29275A043C2D6
:1010CB0080D280D29275A046C280D280C283D28356
:1010DB00C29275A044C280D280D29275A023C280E6
:1010EB00D280C283D283C29275A045C280D280D2F5
:1010FB009275A076C280D280C283D283C29275A031
:10110B0046C280D280D29275A000C280D280C283A8
:10111B00D283C29275A047C280D280D29275A05E54
:10112B00C280D280C283D283C29275A048C280D2C1
:10113B0080D29275A04FC280D280C283D283C292DA
:10114B0075A049C280D280D29275A040C280D28055
:10115B00C283D283C29275A017C280D280D29275FD
:10116B00A061C280D280C283D283C29275A02BC2EF
:10117B0080D280D29275A0F9C280D280C283D283F2
:10118B00C29275A01BC280D280D29275A014C2806D
:10119B00D280C283D283C29275A01AC280D280D26F
:1011AB009275A011C280D280C283D283C29275A0E5
:1011BB001CC280D280D29275A00DC280D280C28315
:1011CB00D283C29275A01FC280D280D29275A03DED
:1011DB00C280D280C283D283C29275A019C280D240
:1011EB0080D29275A00AC280D280C283D283C2926F
:1011FB0075A019C280D280D29275A01AC280D280FB
:10120B00C283D283C29275A019C280D280D292754A
:10121B00A012C280D280C283D283C29275A01EC29A
:10122B0080D280D29275A020C280D280C283D2831A
:10123B00C29275A03CC280D280D29275A060C2804F
:10124B00D280C283D283C29275A03DC280D280D29B
:10125B009275A040C280D280C283D283C29275A005
:10126B0034C280D280D29275A038C280D280C28321
:10127B00D283C29275A035C280D280D29275A0382B
:10128B00C280D280C283D283C29275A024C280D284
:10129B0080D29275A038C280D280C283D283C29290
:1012AB0075A024C280D280D29275A03CC280D2801D
:1012BB00C283D283C29275A016C280D280D292759D
:1012CB00A01CC280D280C283D283C29275A001C2FD
:1012DB0080D280D29275A006C280D280C283D28384
:1012EB00C29275A055C280D280D29275A000C280E6
:1012FB00D280C283D283C29275A002C280D280D226
:10130B009275A000C280D280C283D283C29275A094
:10131B0003C280D280D29275A000C280D280C283D9
:10132B00D283C29275A004C280D280D29275A000E3
:10133B00C280D280C283D283C29275A005C280D2F2
:10134B0080D29275A0EFC280D280C283D283C29228
:10135B0075A006C280D280D29275A000C280D280C6
:10136B00C283D283C29275A007C280D280D29275FB
:10137B00A000C280D280C283D283C29275A008C261
:10138B0080D280D29275A001C280D280C283D283D8
:10139B00C29275A009C280D280D29275A08FC280F2
:1013AB00D280C283D283C29275A022C280D280D255
:1013BB0092C28375A60075A0FF2275A6FFD283C2C9
:1013CB009275A003C280D280D29289A0C280D280B3
:1013DB00C283D283C29275A006C280D280D292EB16
:1013EB00F5A0C280D280C283D283C29275A007C2FD
:1013FB0080D280D292EAF5A0C280D280C283D283FF
:10140B00C29275A022C280D280D292C2832274F77C
:10141B00120E007409120DE1E0F508A3E0F509D2F4
:10142B0083C29275A002C280D280D29275A000C2F4
:10143B0080D280C283D283C29275A003C280D28035
:10144B00D29289A0C280D280C283D283C29275A06D
:10145B0004C280D280D29275A000C280D280C28397
:10146B00D283C29275A005C280D280D2928CA0C2C8
:10147B0080D280C283D283C29275A006C280D280F2
:10148B00D292EBF5A0C280D280C283D283C2927576
:10149B00A007C280D280D292EAF5A0C280D280C2CD
:1014AB0083D283C29275A008C280D280D292E50902
:1014BB00F5A0C280D280C283D283C29275A009C22A
:1014CB0080D280D292E508F5A0C280D280C283D2AE
:1014DB0083C29275A022C280D280D292C28302357F
:1014EB005974F5120E00740B120DE1E0F50AA3E02E
:1014FB00F50B7E987F9E75A6FF780A120EA6121426
:10150B00197402120DACD283C29275A022C280D282
:10151B0080D292C283900902E0FAA3E0D283FC8CC2
:10152B00A0C280D280EAF5A0C280D280C283D283CF
:10153B008CA0C280D280F5A0C280D280C283EEF88C
:10154B00EFF9E824FF1EE934FFFFE84970C7750A7D
:10155B008F750B01780A120EA67CEF7A007B00794F
:10156B00001214197402120DAC7F04020E6674F88B
:10157B00120E00EAFEEBFFD29675A6FF7A007B00F7
:10158B0079001213C5D283C29275A022C280D28079
:10159B00D292C2837AF97BC0EFF8D28388A0C28043
:1015AB00D280EEF5A0C280D280C283D28388A0C243
:1015BB0080D280F5A0C280D280C283EAF974FF2961
:1015CB001A0470D6EBFC74FF2C1B0470CD0226D9C9
:1015DB0074F2120E00890D8C08743B2508F5827489
:1015EB00843400F583E493900901F0F50875090044
:1015FB0074037808120D839008FFE508F0A3E50942
:10160B00F08A088B09EA2408FEEB3400FF9008FFF0
:10161B00E0F8A3E0F9E8C333F8E933F9743B28F5B4
:10162B000A747A39F50BAA08AB09A90D1213C57800
:10163B00007920D283C29275A022C280D280D2922E
:10164B00C283750E0E850A82850B83E49358FAA329
:10165B00E49359FBEA4B6012900904E0FAA3E0D241
:10166B0083F5A0C280D280EA8010900906E0FCA32B
:10167B00E0D283F5A0C280D280ECF5A0C280D280EC
:10168B00C283E9C313F9E813F8150EE50E70B6E53E
:10169B000A2402F50AE50B3400F50BE5082401F5E5
:1016AB0008E5093400F509EE65087003EF6509607C
:1016BB00030216317F07020E6674F1120E00890FBA
:1016CB008C088A0A8B0BEA2456FEEB3401FF750C4F
:1016DB008B750D6FEDF50EAA0AAB0BA90F1213C587
:1016EB00D283C29275A022C280D280D292C283854D
:1016FB000C82850D83E5822408F8E5833400F97BA1
:10170B00807A08E4935BD283600D850EA0C280D2F1
:10171B0080E508F5A0800A75A074C280D28075A000
:10172B0053C280D280C283EBC313FB1AEA70D4A3DB
:10173B00E865827003E9658370C5E50C2408F50C38
:10174B00E50D3400F50DE50A2401F50AE50B34002F
:10175B00F50BEE650A7003EF650B60030216E28072
:10176B0004C296D2967F08020E6674F8120E009091
:10177B000902E0F8A3E0F9900906E8F0A3E9F0907C
:10178B00090874BFF0A3741DF090090474FFF0A353
:10179B00F0900902E0FAA3E0FB1215799008FBE048
:1017AB00D2E0F07C8F7D017A017B00791212190156
:1017BB007C8F7D017A017B0079011219017C8F7D71
:1017CB00017A017B0079DF1219017C8F7D017A018F
:1017DB007B0079EF1219017E007F0075824D7583B6
:1017EB00098019EEFAEFFBEA75F00AA4FAA8F07576
:1017FB00F00AEBA428FB79021215DBA3E0FCEE2424
:10180B00010EEF3400FF743F6C70D87E007F0075C3
:10181B0082757583098019EEFAEFFBEA75F00AA45D
:10182B00FAA8F075F00AEBA428FB79E11215DBA3FB
:10183B00E0FCEE24010EEF3400FF743F6C70D89087
:10184B000B5CE0F8A3E0F9900904E8F0A3E9F0756C
:10185B00829D7583097EC87F008012EEFAEFFB79BB
:10186B00021215DBEE240AFEEF3400FFA3E0FC743A
:10187B003F6C70E77582A67583097E407F018012ED
:10188B00EEFAEFFB79E11215DBEE240AFEEF3400E2
:10189B00FFA3E0FC743F6C70E7900B5EE0F8A3E0F5
:1018AB00F9900904E8F0A3E9F07582A67583097E27
:1018BB005E7F018012EEFAEFFB79E11215DBEE246D
:1018CB000AFEEF3400FFA3E0FC743F6C70E77582F7
:1018DB009D7583097E2C7F018012EEFAEFFB790256
:1018EB001215DBEE240AFEEF3400FFA3E0FC743F7D
:1018FB006C70E70226D974F6120E00890A8A088BDF
:10190B0009ECFEEDFF1213C59008FBE0A2E0E433F7
:10191B00600514602C8067900908E0FAA3E0D2837D
:10192B00F5A0C280D280EAF5A0C280D280C283EE3D
:10193B00F8EFF9E824FF1EE934FFFFE84970D8807F
:10194B003D900908E0FAA3E0D283F5A0C280D280D3
:10195B00EAF5A0C280D280C283AA08AB09A90A12F9
:10196B0013C5E5082401F508E5093400F509EEF87F
:10197B00EFF9E824FF1EE934FFFFE84970C37F034A
:10198B00020E6674F7120E0090090874EFF0A37440
:10199B007BF07508197509007E147F00AA08AB0946
:1019AB00EEF91213C5900908E0FAA3E0D283F5A073
:1019BB00C280D280EAF5A0C280D280C283EE240519
:1019CB00FEEF3400FFC3EE94E0EF940040CEE50849
:1019DB002419F508E5093400F509C3E508948FE5EA
:1019EB0009940140B37508147509007E007F00EE61
:1019FB00FAEFFBA9081213C5900908E0FAA3E0D28D
:101A0B0083F5A0C280D280EAF5A0C280D280C283C7
:101A1B00EE2405FEEF3400FFC3EE948FEF940140EC
:101A2B00CEE5082419F508E5093400F509C3E508E6
:101A3B0094E0E509940040B39008FBE0C2E0F07C31
:101A4B00C87D007AC87B007914121901E0D2E0F04E
:101A5B007C8F7D017A007B00797802355674F71202
:101A6B000E00900908E0F508A3E0F509900902E0E3
:101A7B00F8A3E0F9900908E8F0A3E9F0900906E86B
:101A8B00F0A3E9F09008FBE0C2E0F07E127F007C4F
:101A9B000D7D00EEFAEFFB79021219017C0D7D0032
:101AAB00EE2401FAEF3400FB7902121901EE240A3D
:101ABB00FEEF3400FF74AC6E700374016F70D0E0F6
:101ACB00C2E0F07E127F007C0D7D00EEFAEFFB7919
:101ADB00E11219017C0D7D00EE2401FAEF3400FBBD
:101AEB0079E1121901EE240AFEEF3400FF74AC6E9B
:101AFB00700374016F70D074026521700990090432
:101B0B0074FFF0A3801EE5217005900B5C800974B7
:101B1B000165217010900B5EE0F8A3E0F9900904C9
:101B2B00E8F0A3E9F07582F775830A7E147F0080D5
:101B3B0012EEFAEFFB79021215DBEE240AFEEF34FC
:101B4B0000FFA3E0FC743F6C70E7900B5CE0F8A324
:101B5B00E0F9900904E8F0A3E9F075820B75830BAB
:101B6B007EBE7F008012EEFAEFFB79021215DBEEE0
:101B7B00240AFEEF3400FFA3E0FC743F6C70E79087
:101B8B000B5EE0F8A3E0F9900904E8F0A3E9F07527
:101B9B00821575830B7E227F018012EEFAEFFB79A3
:101BAB00021215DBEE240AFEEF3400FFA3E0FC74F7
:101BBB003F6C70E79008F9E0A2E7900904500874B5
:101BCB00E0F0A37407800474FFF0A3F0758229750D
:101BDB00830B7E5A7F008012EEFAEFFB79E1121530
:101BEB00DBEE240AFEEF3400FFA3E0FC743F6C70C5
:101BFB00E7E5217011900B5CE0F8A3E0F990090484
:101C0B00E8F0A3E98012740165217005900B5E80EA
:101C1B00E790090474FFF0A3F075821F75830B7EA8
:101C2B00147F008012EEFAEFFB79E11215DBEE2444
:101C3B000AFEEF3400FFA3E0FC743F6C70E79009E1
:101C4B000474FFF0A3F075820175830B7E5A7F003D
:101C5B008012EEFAEFFB79021215DBEE240AFEEF8F
:101C6B003400FFA3E0FC743F6C70E775823375831F
:101C7B000B7E967F008012EEFAEFFB79E11215DBFB
:101C8B00EE240AFEEF3400FFA3E0FC743F6C70E718
:101C9B0075823D75830B7EE67F008012EEFAEFFBBB
:101CAB0079E11215DBEE240AFEEF3400FFA3E0FC12
:101CBB00743F6C70E7900B5CE0F8A3E0F9900904BB
:101CCB00E8F0A3E9F09008F4E070257582AA75831B
:101CDB00097E367F01E0FC743F6C6039EEFAEFFB56
:101CEB0079E11215DBEE240AFEEF3400FFA380E549
:101CFB007582B07583097E367F018012EEFAEFFB99
:101D0B0079E11215DBEE240AFEEF3400FFA3E0FCB1
:101D1B00743F6C70E7900B5EE0F8A3E0F990090458
:101D2B00E8F0A3E9F09008F4E070257582AA7583BA
:101D3B00097E547F01E0FC743F6C6039EEFAEFFBD7
:101D4B0079E11215DBEE240AFEEF3400FFA380E5E8
:101D5B007582B07583097E547F018012EEFAEFFB1A
:101D6B0079E11215DBEE240AFEEF3400FFA3E0FC51
:101D7B00743F6C70E7900908E508F0A3E509F002E1
:101D8B003559C082C0839008E77401F09008FCE0DD
:101D9B004412F07959121E89900AF5E09008D3F09D
:101DAB009008E7E09008D4F09008E8E09008D5F0B0
:101DBB009008E9E09008D6F09008E77402F09008DC
:101DCB00FCE04412F07959121E899008E7E0900864
:101DDB00D7F09008E8E09008D8F09008E9E0900878
:101DEB00D9F09008E77408F09008FCE04412F07901
:101DFB0059121E899008E7E09008DAF09008E8E0A5
:101E0B009008DBF09008E9E09008DCF09008E774AC
:101E1B000EF09008FCE0C2E1F0D2E4F07959121E0A
:101E2B00899008E7E09008DDF09008E8E09008DE84
:101E3B00F09008E77437F09008FCE0C2E1F0D2E4D0
:101E4B00F07959121E899008E7E09008DFF09008AE
:101E5B00E8E09008E0F09008E7740DF09008FCE0E3
:101E6B00C2E1F0D2E4F07959121E899008E7E090B4
:101E7B0008E1F09008E8E09008E2F0021F14C0823D
:101E8B00C0837A007B00A2A8E433F8C2A8E9900AC9
:101E9B00F5F0E8333333F89008FCE054F74844018D
:101EAB00F0A2E45007C2E4F0D2E28002C2E2F0D228
:101EBB00C5E0A2E0501CEAFCEBFDEC24010AED347A
:101ECB0000FBC3EC94E9ED94FD40EBE0C2E0F0C302
:101EDB0040E49008FEE0A2E25027E0A2E14022900D
:101EEB0008E8E4F09008E9F09008E704F09008FCAB
:101EFB00E0C2E2F0D2C5A2E040FC9008FEE0C2E2F4
:101F0B00F09008FCE0A2E392A8D083D08222C0E03C
:101F1B00C0D0E8C0E0E9C0E0C082C083A298400313
:101F2B0002210A9008CAE070079008CDE4F0A3F0F4
:101F3B00C298E5999008D2F09008CAE0C39411407A
:101F4B000302216C9008D2E0C0E09008CDE024BAE7
:101F5B00F8A3E03408F988828983D0E0F09008CAAE
:101F6B00E004F09008CDE02401F0A3E03400F09001
:101F7B0008CAE06410600302216C9008C9E0640D8C
:101F8B0060030220F19008C8E0F89008F9E0A2E5A0
:101F9B00500A740A68700543EF1080239008ECE038
:101FAB0064017005740A6860EE740F68700790081E
:101FBB00ED74018009740A6860F79008EDE4F09005
:101FCB0008F9C0829008BAE0A2E0758308D082E0DD
:101FDB0092E3F09008F9C0829008BBE0A2E0758311
:101FEB0008D082E092E1F09008F9C0829008BCE042
:101FFB00A2E0758308D082E092E2F09008F9E0A2AB
:10200B00E1400DE0A2E240089008BDE09008F0F03E
:10201B009008BEE09008E8F09008BFE09008E9F067
:10202B009008C0E09008E7F09008C1E0900AF5F046
:10203B009008C2E0900AF6F09008C3E09008D1F047
:10204B009008F9C0829008C4E0A2E0758308D082A2
:10205B00E092E6F09008D1E064017004C2B0800217
:10206B00D2B09008BAE0602A64027008900AF6E0D9
:10207B00F5FC800BE064037006900AF6E0F5EAC20B
:10208B00969008EEE4F0A3F0D2969008F9E0C2E047
:10209B0080109008F9E0A2E140F3E0A2E240EEE00C
:1020AB00D2E0F09008E7E0640170089008FCE0D201
:1020BB00E18010E0640260F3E0640860EE9008FCDD
:1020CB00E0C2E1F09008C7E0600F9008F9E0C2E0D1
:1020DB00F09008FAE0D2E380069008FAE0C2E3F051
:1020EB009008CAE4807A9008CAE4F09008F9E0D22C
:1020FB00E0F0E0C2E3F0E0C2E1F0E0C2E28061A216
:10210B0099505EC299900AF3E0F8A3E0F9E8499080
:10211B0008CB6040E0687003A3E06970079008CFBC
:10212B00E4F0A3F09008CFE024A5F8A3E03401F984
:10213B0088828983E09008D2F0F5999008CFE0244B
:10214B0001F0A3E03400F0900AF3E024FFF0A3E0E9
:10215B0034FF800CE0F8A3E0F9900AF3E8F0A3E970
:10216B00F0D083D082D0E0F9D0E0F88004D083D0D7
:10217B0082D0D0D0E032C0E0C0D0C082C083A2C237
:10218B0050030222CFE5C054F02480700302229545
:10219B0024C0602124E060030222CF900AF5E0C343
:1021AB0033F5C253C2FE9008FCE0A2E4E43342C212
:1021BB00C2C50222CFA2C140030222849008FCE0D8
:1021CB00A2E450030222CF9008EAE064017023904E
:1021DB000AF5E0645D600AE064486005E0644970FC
:1021EB00679008FCE0C2E0F09008EAE4F0D2C40289
:1021FB0022CF9008FCE0A2E140319008EAE06402B3
:10220B007029900AF5E0645070D79008FCE0A2E2C8
:10221B00505C900AF5E0645070549008FCE0D2E4F6
:10222B00F0D2C59008EA74010222CE9008EAE06071
:10223B000C1460141460D31460A70222CF7401F045
:10224B009008E7E0F5C2807C9008FCE0A2E2501316
:10225B00900AF5E06450600B9008FCE0D2E4F0D2F9
:10226B00C580619008EA7402F09008E880D5900868
:10227B00EA7403F09008E980CA9008EAE4F0D2C44B
:10228B00900AF5E0645D603C80D59008EAE014604C
:10229B000514601A802EE5C29008E8F09008EA74E5
:1022AB0002F09008FCE0A2E1500AD2C18016E5C210
:1022BB009008E9F0C2C1D2C49008EAE4F09008FC9F
:1022CB00E0C2E0F0C2C0022178C0E0C0D0C082C042
:1022DB0083D2909008F9E0D2E4F0022178C0E0C0FC
:1022EB00D0E8C0E0C082C083900B62E0F874012894
:1022FB00F0E8C39405406B75A60075A0FFC296C2AB
:10230B00839008FDA2A5E092E0F0A2A0E092E1F09C
:10231B00A2A6E092E2F0A2A7E092E3F0A2A2E092E2
:10232B00E4F0A2A1E092E5F0A2A3E092E6F0A2A471
:10233B00E092E7F0E0F460239008FEE0A2E4401B9B
:10234B009008FAE0A2E45005E0D2E5800D9008FE7B
:10235B00E0D2E3F09008F9E0C2E3F0D296900B6282
:10236B00E4F0C2CFD083D08202217374F8120E0036
:10237B009008E7E4F09008E8F09008FCE0C2E1F088
:10238B00D2E4F07950121E899008E8E0F523D2AD23
:10239B00900B62E060FAC2AD74EE652370347F017E
:1023AB007E249008E7E4F0EF9008E8F09008FCE05A
:1023BB00C2E1F0D2E4F07950121E899008E8E0C037
:1023CB00E0EEF8D0E0F6D2ADC2AD0F0EEFC3941431
:1023DB0040D0E524FAC333F8E433F9743B28F58293
:1023EB00748039F583E493F8740193F9900B5CE8EE
:1023FB00F0A3E9F0E525FBC333F8E433F9743B288C
:10240B00F582748039F583E493F8740193F9900B9A
:10241B005EE8F0A3E9F0E526FCC333F8E433F97486
:10242B003B28F582748239F583E493F8740193F9B0
:10243B00900902E8F0A3E9F0EA900AEFF0A3E4F0C8
:10244B00EB9008B3F0A3E4F0EC9008B5F0A3E4F044
:10245B00D2AD0226D974F2120E00890A8C0B7EFFC4
:10246B007F007508017509F87402650B70048F08FD
:10247B008F0975A6FFEA2400F50CEB3401F50D78F6
:10248B000C120EA67414250AFC1214197402120DE8
:10249B00ACD283C29275A022C280D280D292C28368
:1024AB007A3B7B807C3B7D82750C14750D00E509B6
:1024BB00F50ED283850EA0C280D280E508F5A0C2AE
:1024CB0080D280C283A80CA90DE824FFF50CE93457
:1024DB00FFF50DE84970DB7402650B60068A828B91
:1024EB008380048C828D83E493C0E0740193F58325
:1024FB00D0828582088583098E0C8F0DE50C24FF15
:10250B001EE50D34FFFFEC24020C0CED3400FDEA4C
:10251B002402EB34000A0AFBE50C450D708A021607
:10252B00BF74F5120E00E9FE7FFF900912E004F074
:10253B0075A6FF7508007509017808120EA67C3286
:10254B00900912E0FA7B0079281214197402120D0B
:10255B00ACD283C29275A022C280D280D292C283A7
:10256B007C0AEE70307C0A900902E0FAA3E0D28379
:10257B00F5A0C280D280EAF5A0C280D280C2838C43
:10258B000874FF25081C0470DE8F0974FF25091FD2
:10259B000470D2801BD28375A000C280D28075A03C
:1025AB001FC280D280C283ECFF74FF2F1C0470E526
:1025BB0002155974F8120E00900902E0F8A3E0F925
:1025CB00900906E8F0A3E9F0900B5CE0F8A3E0F9C2
:1025DB00900904E8F0A3E9F07582B67583097E14BF
:1025EB007F008012EEFAEFFB79BE1215DBEE240AA8
:1025FB00FEEF3400FFA3E0FC743F6C70E7900B5EC2
:10260B00E0F8A3E0F9900904E8F0A3E9F07582C2C1
:10261B007583097E147F008012EEFAEFFB79A0120E
:10262B0015DBEE240AFEEF3400FFA3E0FC743F6CD5
:10263B0070E790090474FFF0A3F07582CE758309DF
:10264B007E147F008012EEFAEFFB79821215DBEE1F
:10265B00240AFEEF3400FFA3E0FC743F6C70E775B7
:10266B0082DA7583097E147F008012EEFAEFFB7914
:10267B005F1215DBEE240AFEEF3400FFA3E0FC74BF
:10268B003F6C70E77582F07583097E147F008012B2
:10269B00EEFAEFFB793C1215DBEE240AFEEF340069
:1026AB00FFA3E0FC743F6C70E77582FF7583097EB6
:1026BB00147F008012EEFAEFFB791E1215DBEE246D
:1026CB000AFEEF3400FFA3E0FC743F6C70E77F0160
:1026DB00020E6674F8120E00900902E0F8A3E0F9FE
:1026EB00900908E8F0A3E9F0900906E8F0A3E9F0F7
:1026FB009008FBE0C2E0F07E127F007C0D7D00EEC7
:10270B00FAEFFB79BE1219017C0D7D00EE2401FA64
:10271B00EF3400FB79BE121901EE240AFEEF3400F0
:10272B00FF74806E7001EF70D2E0C2E0F07E127F1A
:10273B00007C0D7D00EEFAEFFB79A01219017C0DE8
:10274B007D00EE2401FAEF3400FB79A0121901EEA3
:10275B00240AFEEF3400FF74806E7001EF70D2E03C
:10276B00C2E0F07E127F007C0D7D00EEFAEFFB796C
:10277B00821219017C0D7D00EE2401FAEF3400FB6F
:10278B007982121901EE240AFEEF3400FF74806E79
:10279B007001EF70D2E0C2E0F07E127F007C0D7D05
:1027AB0000EEFAEFFB795F1219017C0D7D00EE2430
:1027BB0001FAEF3400FB795F121901EE240AFEEFE8
:1027CB003400FF74E46E7001EF70D2E0C2E0F07E73
:1027DB00127F007C0D7D00EEFAEFFB793C121901A4
:1027EB007C0D7D00EE2401FAEF3400FB793C1219CD
:1027FB0001EE240AFEEF3400FF749E6E7001EF7041
:10280B00D2E0C2E0F07E127F007C0D7D00EEFAEF8D
:10281B00FB791E1219017C0D7D00EE2401FAEF34B9
:10282B0000FB791E121901EE240AFEEF3400FF742F
:10283B00C66E7001EF70D21225BE0226D974F71244
:10284B000E00C2A8C2ACC2AD900902E0F8A3E0F939
:10285B00900906E8F0A3E9F075088F75090178086F
:10286B00120EA67CDE7A007B0079141214EC740233
:10287B00120DAC1225BE7C007A8C7B0079B9122428
:10288B00607C017A8C7B00799B1224607C027A8CB1
:10289B007B00797D1224607808120EA67CEF7A00FB
:1028AB007B0079001214197402120DAC9009087494
:1028BB00FFF0A3F09008FBE0C2E0F07C057D0090F8
:1028CB000AEFE0248CFAA3E03400FB79CE12190155
:1028DB007C057D009008B3E0248CFAA3E03400FB68
:1028EB0079B01219017C057D009008B5E0248CFAB3
:1028FB00A3E03400FB799202355674F8120E00C235
:10290B00AD9008FAE0C2E5F09008FDE0F8E0A2E631
:10291B00E43344FEF4F9E8A2E7E43344FEF490090F
:10292B000AF8E028C399F0F4700474058007E0C33B
:10293B0094064002E4F090090BE0F890090AE06875
:10294B0060031226DEE06021147003022A07147064
:10295B0003022A9A147003022B2D147003022BC34B
:10296B00147003022D0C022DD47A00900AEFE0F9BB
:10297B00122DDF900B5CEAF0A3EBF0900B5CE0F810
:10298B00A3E0F9900908E8F0A3E9F0900906E8F054
:10299B00A3E9F090090474FFF0A3F09008FBE0C2E8
:1029AB00E0F07E127F007C0D7D00EEFAEFFB79BE2E
:1029BB001219017C0D7D00EE2401FAEF3400FB7936
:1029CB00BE121901EE240AFEEF3400FF74806E7004
:1029DB0001EF70D27582B67583097E147F00E0FC1F
:1029EB00743F6C7003022DD4EEFAEFFB79BE121517
:1029FB00DBEE240AFEEF3400FFA380E27A0190089D
:102A0B00B3E0F9122DDF900B5EEAF0A3EBF0900B25
:102A1B005EE0F8A3E0F9900908E8F0A3E9F090096B
:102A2B0006E8F0A3E9F090090474FFF0A3F0900816
:102A3B00FBE0C2E0F07E127F007C0D7D00EEFAEF32
:102A4B00FB79A01219017C0D7D00EE2401FAEF3405
:102A5B0000FB79A0121901EE240AFEEF3400FF747B
:102A6B00806E7001EF70D27582C27583097E147F00
:102A7B0000E0FC743F6C7003022DD4EEFAEFFB798F
:102A8B00A01215DBEE240AFEEF3400FFA380E27ADE
:102A9B00029008B5E0F9122DDF900902EAF0A3EBE2
:102AAB00F0900902E0F8A3E0F9900908E8F0A3E937
:102ABB00F0900906E8F0A3E9F090090474FFF0A385
:102ACB00F09008FBE0C2E0F07E127F007C0D7D00F1
:102ADB00EEFAEFFB79821219017C0D7D00EE2401D9
:102AEB00FAEF3400FB7982121901EE240AFEEF345F
:102AFB0000FF74806E7001EF70D27582CE75830902
:102B0B007E147F00E0FC743F6C7003022DD4EEFA50
:102B1B00EFFB79821215DBEE240AFEEF3400FFA3E4
:102B2B0080E2900B60E0F8A3E0F9900908E8F0A3CD
:102B3B00E9F0900906E8F0A3E9F090090474FFF0BE
:102B4B00A3F09008FBE0C2E0F07E127F007C0D7DCD
:102B5B0000EEFAEFFB795F1219017C0D7D00EE247C
:102B6B0001FAEF3400FB795F121901EE240AFEEF34
:102B7B003400FF74E46E7001EF70D27582DA7583E6
:102B8B00097E147F008012EEFAEFFB795F1215DBE2
:102B9B00EE240AFEEF3400FFA3E0FC743F6C70E7F9
:102BAB009008FDE0A2E45008E0A2E55003022DD40A
:102BBB007900122EDE022DD4900B60E0F8A3E0F921
:102BCB00900908E8F0A3E9F0900906E8F0A3E9F012
:102BDB0090090474FFF0A3F09008FBE0C2E0F07ED4
:102BEB00127F007C0D7D00EEFAEFFB793C12190190
:102BFB007C0D7D00EE2401FAEF3400FB793C1219B9
:102C0B0001EE240AFEEF3400FF749E6E7001EF702C
:102C1B00D27582F07583097E147F008012EEFAEF75
:102C2B00FB793C1215DBEE240AFEEF3400FFA3E028
:102C3B00FC743F6C70E79008FDE0A2E45008E0A242
:102C4B00E55003022DD49008FAE0C2E4F07523EEB0
:102C5B00900AEFE0F5249008B3E0F5259008B5E075
:102C6B00F5269008E7E4F09008E8F09008E974EE98
:102C7B00F09008FCE0C2E4F0D2E1F07950121E892A
:102C8B00D2AD900B62E060FAC2AD7F017E2490085A
:102C9B00E7E4F0EF9008E8F0EEF8E69008E9F09042
:102CAB0008FCE0C2E4F0D2E1F07950121E89D2ADFB
:102CBB00C2AD0F0EEFC3940440D4D2AD900B63E0C2
:102CCB00603C900B64E06036D2ADC2AD7F047E27D2
:102CDB009008E7E4F0EF9008E8F0EEF8E69008E9EA
:102CEB00F09008FCE0C2E4F0D2E1F07950121E89BA
:102CFB00D2ADC2AD0F0EEFC3941440D4D2AD022DA2
:102D0B00CE900B60E0F8A3E0F9900908E8F0A3E996
:102D1B00F0900906E8F0A3E9F090090474FFF0A322
:102D2B00F09008FBE0C2E0F07E127F007C0D7D008E
:102D3B00EEFAEFFB791E1219017C0D7D00EE2401DA
:102D4B00FAEF3400FB791E121901EE240AFEEF3460
:102D5B0000FF74C66E7001EF70D27582FF75830928
:102D6B007E147F008012EEFAEFFB791E1215DBEE5C
:102D7B00240AFEEF3400FFA3E0FC743F6C70E79075
:102D8B0008FDE0A2E45005E0A2E5403D9008FAE022
:102D9B00C2E4F090090CE0F8A3E0F9900B5CE8F0CA
:102DAB00A3E9F090090EE0F8A3E0F9900B5EE8F0D0
:102DBB00A3E9F0900910E0F8A3E0F9900902E8F01C
:102DCB00A3E9F0D2A8D2ACC2AD90090AE090090BEE
:102DDB00F00226D974F8120E00E9FEEAFF90090200
:102DEB00E0F8A3E0F9900908E8F0A3E9F09008FBFC
:102DFB00E0C2E0F07C057D00900AEFE0248CFAA3A2
:102E0B00E03400FB79CE1219017C057D009008B3EC
:102E1B00E0248CFAA3E03400FB79B01219017C0595
:102E2B007D009008B5E0248CFAA3E03400FB799286
:102E3B001219019008FDE0A2E440030E8006E0A207
:102E4B00E540011E90090874FFF0A3F0EF60081431
:102E5B00600B14600E8014EE900AEF800AEE90085F
:102E6B00B38004EE9008B5F0A3E4F07C057D0090F0
:102E7B000AEFE0248CFAA3E03400FB79CE1219019F
:102E8B007C057D009008B3E0248CFAA3E03400FBB2
:102E9B0079B01219017C057D009008B5E0248CFAFD
:102EAB00A3E03400FB7992121901EEC333F8E4333B
:102EBB00F974026F7009743B28F582748280077471
:102ECB003B28F582748039F583E493FA740193FB04
:102EDB000226D974F7120E00900B637401F0900B5D
:102EEB0064F0900AF1E4F0900AF2F0900906F0A376
:102EFB00F075088F7509017808120EA67CDE7A0032
:102F0B007B0079141214EC7402120DAC900904744A
:102F1B00FFF0A3F0900902E0F8A3E0F9900906E8AE
:102F2B00F0A3E9F07808120EA67CDE7A007B00791C
:102F3B00141214EC7402120DAC75821275830A7E96
:102F4B00147F008012EEFAEFFB79BE1215DBEE2434
:102F5B000AFEEF3400FFA3E0FC743F6C70E7758250
:102F6B001D75830A7E147F008012EEFAEFFB79AA9F
:102F7B001215DBEE240AFEEF3400FFA3E0FC743FD6
:102F8B006C70E7900912E4F0900AF18022900AF13C
:102F9B00E0F8741528F58274093400F583E0C0E07D
:102FAB00900AF1E02427F8D0E0F6900AF1E004F063
:102FBB00E0C39408400302319B790012252C900941
:102FCB0012E4F0FC78AD79088C08900AF1E075F00A
:102FDB0005A4FAABF074612AFA74893BFBEA250865
:102FEB00F582EB3400F583E49388828983F00CA39C
:102FFB00A882A983ECC3940540CE7582AD75830876
:10300B007E507F008012EEFAEFFB79AA1215DBEEF1
:10301B00240AFEEF3400FFA3E0FC743F6C70E790D2
:10302B000AF1E0FEC394059008EBE04004C2E08097
:10303B0002D2E0F09008FCE054EDF09008EBE09049
:10304B0008E7F0795D121E899008FCE054EDF0EE74
:10305B00C333F8E433F974B128F582748939F583F5
:10306B00E4939008E7F07948121E897E0090091DC1
:10307B00E4F0790112252C8EEA7F2812355E1FEFC2
:10308B0070F912355E900913E02483C39407400353
:10309B00023124E5EAC0E0900AF1E0F8741528F556
:1030AB008274093400F583D0E0F090091D7401F0AF
:1030BB0075F014900AF1E0A4F874BE98F5087582C7
:1030CB002575830A7ED27F008012EEFAEFFBA908EA
:1030DB001215DBEE240AFEEF3400FFA3E0FC743F75
:1030EB006C70E775F014900AF1E0A4F874BE98F5D3
:1030FB00087582AD7583087E2C7F01E0FC743F6CF4
:10310B007003022F98EEFAEFFBA9081215DBEE24E1
:10311B000AFEEF3400FFA380E20E74FF6E60030221
:10312B00307D75F014900AF1E0A4F874BE98F508A0
:10313B0075822A75830A7ED27F008012EEFAEFFB2E
:10314B00A9081215DBEE240AFEEF3400FFA3E0FC06
:10315B00743F6C70E775F014900AF1E0A4F874BE3C
:10316B0098F5087582AD7583087E2C7F018012EE71
:10317B00FAEFFBA9081215DBEE240AFEEF3400FF71
:10318B00A3E0FC743F6C70E7900B63E4F0022FB587
:10319B00900902E0F8A3E0F9900906E8F0A3E9F042
:1031AB0075088F7509017808120EA67CDE7A007BF4
:1031BB000079141214EC7402120DAC758234758301
:1031CB000A7E147F008012EEFAEFFB79BE1215DB3C
:1031DB00EE240AFEEF3400FFA3E0FC743F6C70E7B3
:1031EB0075821D75830A7E147F008012EEFAEFFB49
:1031FB0079AA1215DBEE240AFEEF3400FFA3E0FCE4
:10320B00743F6C70E7900912E4F0900AF280229000
:10321B000AF2E0F8741E28F58274093400F583E095
:10322B00C0E0900AF2E0242FF8D0E0F6900AF2E02A
:10323B0004F0E0C39408400302341D790012252CDE
:10324B00900912E4F0FC78AD79088C08900AF2E052
:10325B0075F005A4FAABF074612AFA74893BFBEAAA
:10326B002508F582EB3400F583E49388828983F09B
:10327B000CA3A882A983ECC3940540CE7582AD75CF
:10328B0083087E507F008012EEFAEFFB79AA1215AD
:10329B00DBEE240AFEEF3400FFA3E0FC743F6C70FE
:1032AB00E7900AF2E0FEC394059008EBE04004C2FD
:1032BB00E18002D2E1F09008FCE054EDF09008EBD5
:1032CB00E09008E7F0795D121E899008FCE054ED60
:1032DB00F0EEC333F8E433F974B128F5827489390D
:1032EB00F583E4939008E7F07949121E897E0090EC
:1032FB000926E4F0790112252C8EFC7F2812355E0D
:10330B001FEF70F912355E900914E02483C3940704
:10331B0040030233A6E5FCC0E0900AF2E0F8741E0D
:10332B0028F58274093400F583D0E0F090092674F7
:10333B0001F075F014900AF2E0A4F874BE98F50849
:10334B0075822575830A7ED27F008012EEFAEFFB21
:10335B00A9081215DBEE240AFEEF3400FFA3E0FCF4
:10336B00743F6C70E775F014900AF2E0A4F874BE29
:10337B0098F5087582AD7583087E2C7F01E0FC748F
:10338B003F6C700302321AEEFAEFFBA9081215DB41
:10339B00EE240AFEEF3400FFA380E20E74FF6E6092
:1033AB00030232FF75F014900AF2E0A4F874BE9891
:1033BB00F50875822A75830A7ED27F008012EEFA99
:1033CB00EFFBA9081215DBEE240AFEEF3400FFA376
:1033DB00E0FC743F6C70E775F014900AF2E0A4F80F
:1033EB0074BE98F5087582AD7583087E2C7F0180BD
:1033FB0012EEFAEFFBA9081215DBEE240AFEEF34EE
:10340B0000FFA3E0FC743F6C70E7900B64E4F002E8
:10341B003237900902E0F8A3E0F9900906E8F0A32F
:10342B00E9F075088F7509017808120EA67CDE7A13
:10343B00007B0079141214EC7402120DAC900B6427
:10344B00E0A2E0C0D0900B63E0A2E092F0120DED91
:10345B00158182F0502875823F75830A7E507F005C
:10346B00E0FC743F6C7003023511EEFAEFFB7978D8
:10347B001215DBEE240AFEEF3400FFA380E2900B63
:10348B0064E0A2E0B392F0900B63E0A2E082F05014
:10349B002575825B75830A7E507F00E0FC743F6C60
:1034AB006064EEFAEFFB79781215DBEE240AFEEF7F
:1034BB003400FFA380E5A2E072F040257582787599
:1034CB00830A7E507F00E0FC743F6C6039EEFAEFAC
:1034DB00FB79781215DBEE240AFEEF3400FFA38094
:1034EB00E575829575830A7E507F008012EEFAEFA8
:1034FB00FB79781215DBEE240AFEEF3400FFA3E014
:10350B00FC743F6C70E77582AE75830A7E287F0072
:10351B008012EEFAEFFB79281215DBEE240AFEEF90
:10352B003400FFA3E0FC743F6C70E79008FD74FF60
:10353B00F0D2ADE0F460FC9008FEE0C2E4F0C2AD66
:10354B009008FD74FFF012284880031219017F02C6
:10355B00020E6674F1120E0074FC120D96900B6540
:10356B007808120C75900B65120C938510828511DF
:10357B0083120C9FC2ADD2A8C290D297D29590085D
:10358B00F9E0A2E450F8E0C2E4F0C2A8D29075A62C
:10359B000075A0FF7464C297D297C295D295147030
:1035AB00F57A2C7B01C29785A00C743B250CF58218
:1035BB0074863400F583E493F50CE4F50DF50EF504
:1035CB000F7808790C120C4FD297C29585A00C740A
:1035DB003B250CF58274863400F583E493F50C855A
:1035EB001082851183780C120C62D295EA24FF1A93
:1035FB00EB34FFFBEA4B70AD900B69780C120C753A
:10360B007808790C120BFDE508900913F0851082F0
:10361B008511837808120C75900B69780C120C7558
:10362B007808790C120BFDE508900914F0C296D2BC
:10363B009675A6FF7404120DAC0217709008F9E092
:10364B00D2E5F09008FAE0D2E6F09008FEE0D2E482
:10365B00F09008FD74FFF07521029008FAE0D2E0BB
:10366B00F0E0D2E1F0D2B075245575250075260037
:10367B00120F45E5EFA2E450569008F9E0C2E5F0D1
:10368B00900B65120C939001A1120C9F75A60075FF
:10369B00A0FF9008ECE06401607D900B6D78081240
:1036AB000C759001A17808120C629001A1C0829058
:1036BB000B717808120C75758301D0827808120390
:1036CB005C40C99008F9E0D2E5F09008C8E4F090AE
:1036DB0008F9E0A2E54067120FD8900904E4F0A3C3
:1036EB0074F8F07A007B001215799008FBE0D2E0B9
:1036FB00F07C8F7D017A017B00794F1219017C8F51
:10370B007D017A017B00799F1219017582C975833E
:10371B000A7E9A7F00801A9008F9E0C2E580AFEE2E
:10372B00FAEFFB79701215DBEE240AFEEF3400FF83
:10373B00A3E0FC743F6C70E79008F902384DE0D2BF
:10374B00E5F09008E87418F09008E97440F09008E0
:10375B00E77402F09008FEE0D2E2F09008FCE0C2C1
:10376B00E4F0D2E1F09008FEE0C2E1F07959121ECC
:10377B0089E0D2E2F09008EBE4F09008FCE054ED25
:10378B00F09008EBE09008E7F0795D121E89900845
:10379B00FCE054EDF09008E77408F07948121E89AC
:1037AB009008FCE054EDF09008E77408F0794912AA
:1037BB001E89120FD875A6FF7A537B741215799058
:1037CB0009047437F0A374FFF09009067453F0A347
:1037DB007474F07C377DFF7A237B00795A1216C400
:1037EB007582277583097E1E7F008012EEFAEFFB30
:1037FB0079191215DBEE240AFEEF3400FFA3E0FC6F
:10380B00743F6C70E7D2AD1223769008FDE0F47034
:10381B00089008EDE0640170F19008FEE0C2E4F05E
:10382B00C2AD12177512198E9008F9E0D2E3F09021
:10383B0008FEE0D2E2800EC296D296123B59E0C24D
:10384B00E3F0E0D2E0F09008F9E0A2E55003023992
:10385B007075A60075A0FFE0A2E040FBE0A2E3407C
:10386B00D6E0A2E1501F121D8D900AF37414F0A341
:10387B00E4F09008CB7414F0A3E4F0D2999008F91B
:10388B00E0C2E180BCE0A2E2501D9008FCE0C2E483
:10389B00F0900AF5E0F9121E89900B5B7401F09021
:1038AB0008F9E0C2E2809A9008FAE0A2E350979000
:1038BB0008C6E0F87049A3E0FEC394059008EBE05E
:1038CB004004C2E08002D2E0F09008FCE054EDF03E
:1038DB009008EBE09008E7F0795D121E899008FCE8
:1038EB00E054EDF0EEC333F8E433F974B128F5820C
:1038FB00748939F583E4939008E7F07948804C7428
:10390B000168704AA3E0FEC394059008EBE0400405
:10391B00C2E18002D2E1F09008FCE054EDF0900897
:10392B00EBE09008E7F0795D121E899008FCE054FB
:10393B00EDF0EEC333F8E433F974B128F5827489F2
:10394B0039F583E4939008E7F07949121E899008C2
:10395B00F9E0D2E0F09008FAE0C2E3023850121D11
:10396B008DE0C2E1F09008F9E0A2E54003023B587C
:10397B00800AE0A2E15005C2AD12424ED2AD9008D2
:10398B00F9E0A2E3E0502FA2E75007C2AD1246F2D6
:10399B0080EA9008FAE0F8E0F9E8A2E0500CE9A21E
:1039AB00E15007C2AD1243D780D2E0A2E050C3C2B0
:1039BB00AD1240C580C6A2E140A4E0A2E250219026
:1039CB0008FCE0C2E4F0900AF5E0F9121E89900BB6
:1039DB005B7401F09008F9E0C2E2F0E0D2E380847E
:1039EB009008FEE0A2E340030239709008F9E0C2B0
:1039FB00E2F09008FDE0A2E25003023AA19008EB3E
:103A0B00E06410F09008FCE054EDF09008EBE090CF
:103A1B0008E7F0795D121E89900902E0F8A3E0F93E
:103A2B00900906E8F0A3E9F0900B5CE0F8A3E0F94D
:103A3B00900904E8F0A3E9F09008EBE0A2E4402B36
:103A4B007582A67583097E407F018012EEFAEFFB2B
:103A5B0079E11215DBEE240AFEEF3400FFA3E0FC44
:103A6B00743F6C70E79008F3E4802A7582D67583F7
:103A7B000A7E407F018012EEFAEFFB79E11215DB33
:103A8B00EE240AFEEF3400FFA3E0FC743F6C70E7FA
:103A9B009008F37401F09008FDE0A2E35003023BA1
:103AAB003E9008EBE06420F09008FCE054EDF090C1
:103ABB0008EBE09008E7F0795D121E89900902E0AF
:103ACB00F8A3E0F9900906E8F0A3E9F0900B5EE0AB
:103ADB00F8A3E0F9900904E8F0A3E9F09008EBE013
:103AEB00A2E540257582A67583097E5E7F01E0FC09
:103AFB00743F6C6039EEFAEFFB79E11215DBEE24C3
:103B0B000AFEEF3400FFA380E57582D675830A7E2B
:103B1B005E7F018012EEFAEFFB79E11215DBEE24EA
:103B2B000AFEEF3400FFA3E0FC743F6C70E79008D3
:103B3B00F4E4F0C2AD1248A09008FEE0C2E3F090AE
:103B4B0008F9E0A2E250030239700239E622C08282
:103B5B00C083D2A8C2909008F9E0A2E450F8E0C26A
:103B6B00E4F0C2A8D2909008F0E060046402704BBD
:103B7B009008EEE4F0A3F078A57901D297C297E50F
:103B8B00A088828983F0D2979008EEE02401F0A3FD
:103B9B00E03400F088828983A3A882A9839008EE81
:103BAB00C3E094FFA3E0940140D1D2979001A5E428
:103BBB00F09008CBF0A37402F0D2999008D1E06496
:103BCB00016005E0640270089008F9E0A2E650F885
:103BDB009008F0E064016005E06402704B9008EE21
:103BEB00E4F0A3F078A57901D295C295E5A088827F
:103BFB008983F0D2959008EEE02401F0A3E0340025
:103C0B00F088828983A3A882A9839008EEC3E094ED
:103C1B00FFA3E0940140D19001A57401F09008CB73
:103C2B00E4F0A37402F0D299C296D296021F1474D8
:103C3B00F4120E0075080075A60075A0FF78C57903
:103C4B0004C29785A00A743B250AF582748634005A
:103C5B00F583E49388828983F0D297A3A882A98302
:103C6B00E8B4D503E9640470D875090878CD7904F4
:103C7B00C297E82408FAE93400FB85A00A743B25B7
:103C8B000AF58274863400F583E4938A828B83F081
:103C9B00D297E508A2E0405988828983E0F50CF5BC
:103CAB0082AC82AE12EE24FCF50AE434FFF50BC3B2
:103CBB00E50A9CE50B9400A2D265D0335033EE2479
:103CCB0004FEE43400FFEC9EE49FC365D033502127
:103CDB008A828B83E0FA9008FAE0A2E6500DECC3DF
:103CEB009A500E8509227508018006EAC3950C408F
:103CFB00F2050988828983A3A882A983E509C39465
:103D0B005C5003023C7B0240C074F4120E00750839
:103D1B000075220075A60075A0FF78B97906C295CB
:103D2B0085A00A743B250AF58274863400F583E47A
:103D3B009388828983F0D295A3A882A983E8B4C91A
:103D4B0003E9640670D875090878C17906C295E84D
:103D5B002408FAE93400FB85A00A743B250AF58296
:103D6B0074863400F583E4938A828B83F0D295E5D5
:103D7B0008A2E0405988828983E0F50CF582AC8279
:103D8B00AE12EE24FCF50AE434FFF50BC3E50A9CF6
:103D9B00E50B9400A2D265D0335033EE2404FEE43D
:103DAB003400FFEC9EE49FC365D03350218A828B95
:103DBB0083E0FA9008FAE0A2E6500DECC39A500E9D
:103DCB008509227508018006EAC3950C40F20509A6
:103DDB0088828983A3A882A983E509C3945C5003D5
:103DEB00023D580240C074F2120E007E008E227506
:103DFB00A60075A0FF7AC57B0478B97906C29785B2
:103E0B00A008743B2508F58274853400F583E49390
:103E1B008A828B83F0D297C29585A008743B2508C4
:103E2B00F58274853400F583E49388828983F0D21C
:103E3B0095A3A882A9838A828B83A3AA82AB83E8EA
:103E4B00B4C903E9640670B57F0878CD79047AC1EB
:103E5B007B06C297E82408FCE93400FD85A00874B2
:103E6B003B2508F58274853400F583E4938C828DB1
:103E7B0083F0D297C295EA2408F508EB3400850845
:103E8B000AF50B85A008743B2508F5827485340070
:103E9B00F583E493850A82850B83F0D295EEA2E03D
:103EAB005003023F7FE521706A88828983E0F50E1B
:103EBB00F58285820A851208E50824FCF50CE434AA
:103ECB00FFF50DC3E50C950AE50D9400A2D265D064
:103EDB00334003023F7FE5082404F508E43400F582
:103EEB0009E50A9508E49509C365D0334003023F01
:103EFB007F8C828D83E0FC9008FAE0A2E6500CE503
:103F0B000EC39C506F8F227E018069ECC3950E50BF
:103F1B006380F274016521705B8A828B83E0F50EFE
:103F2B00F582AC82851208E50824FCF50CE434FF1D
:103F3B00F50DC3E50C9CE50D9400A2D265D0335072
:103F4B0033E5082404F508E43400F509EC9508E49E
:103F5B009509C365D033501C850A82850B83E0FC21
:103F6B009008FAE0A2E65006E50EC39C80A1ECC3D4
:103F7B00950E40910F8A828B83A3AA82AB83888292
:103F8B008983A3A882A983EFC3945C5003023E5D8F
:103F9B000216BF74F4120E007C008C2275A60075FD
:103FAB00A0FF78C57904C29785A008743B2508F556
:103FBB008274863400F583E49388828983F0D297E8
:103FCB00C29585A008743B2508F58274863400F5EC
:103FDB0083E49388828983A3F0D295E824020808AE
:103FEB00E93400F9E8B4D503E9640470B97D0878C5
:103FFB00CD7904C297E82408FAE93400FB85A008C0
:10400B00743B2508F58274863400F583E4938A8229
:10401B008B83F0D297C29585A008743B2508F58257
:10402B0074863400F583E49388828983A3A3A3A3C6
:10403B00A3A3A3A3A3F0D295ECA2E0406474026502
:10404B0021605E88828983E0F50CF582AE82851251
:10405B0008E50824FCF50AE434FFF50BC3E50A9EDA
:10406B00E50B9400A2D265D0335036E5082404F555
:10407B0008E43400F509EE9508E49509C365D033DF
:10408B00501F8A828B83E0FA9008FAE0A2E6500B6D
:10409B00EEC39A500C8D227C018006EAC3950C402E
:1040AB00F40D0DE824020808E93400F9EDC3945B24
:1040BB005003023FFE7F05020E6674F1120E00D212
:1040CB00A8C2909008F9E0A2E450F8E0C2E4F0C274
:1040DB00A8D290123C3A74026521700575220180BA
:1040EB0007E522700302424B7E007F00750E297597
:1040FB000F057508A575090185220A74C5250AF5F2
:10410B000C74043400F50D75A60075A0FFC29785DD
:10411B00A00A743B250AF58274863400F583E49378
:10412B00850E82850F83F0D29775A6FF8508828551
:10413B000983E0FC74786C600874C86E7001EF70D2
:10414B000B90090874EFF0A3747B8052EC75F005AB
:10415B0084E5F07012EEF8EFF97A197B00120D1A64
:10416B008B0BEA450B60DAEC2405F8E43400F97AA2
:10417B00197B00120D128B0BEA450B7012EEF8EF48
:10418B00F97A057B00120D1A8B0BEA450B60B29086
:10419B000902E0F8A3E0F9900908E8F0A3E9F0EED2
:1041AB00FAEFFBECF91213C5900908E0FAA3E0D281
:1041BB0083F5A0C280D280EAF5A0C280D280C283F0
:1041CB00900B5CE0F8A3E0F9900908E8F0A3E9F0A4
:1041DB00850C82850D83E024F8F50AEEFAEFFBA936
:1041EB000A1213C5900908E0FAA3E0D283F5A0C226
:1041FB0080D280EAF5A0C280D280C28385088285F6
:10420B000983E50AF0EE24010EEF3400FF850C82E2
:10421B00850D83A385820C85830D85088285098393
:10422B00A3858208858309850E82850F83A38582EA
:10423B000E85830FC3EE948FEF940150030241124E
:10424B0002176C74F1120E00D2A8C2909008F9E01C
:10425B00A2E450F8E0C2E4F0C2A8D290123D14746C
:10426B0002652170057522018007E5227003024368
:10427B00D47E007F00750E1D750F07750835750907
:10428B000385220A74B9250AF50C74063400F50D62
:10429B0075A60075A0FFC29585A00A743B250AF58B
:1042AB008274863400F583E493850E82850F83F048
:1042BB00D29575A6FF850882850983E0FC74786C1E
:1042CB00600874C86E7001EF700B90090874EFF002
:1042DB00A3747B8052EC75F00584E5F07012EEF858
:1042EB00EFF97A197B00120D1A8B0BEA450B60DA8A
:1042FB00EC2405F8E43400F97A197B00120D128BCB
:10430B000BEA450B7012EEF8EFF97A057B00120DF4
:10431B001A8B0BEA450B60B2900902E0F8A3E0F9A7
:10432B00900908E8F0A3E9F0EEFAEFFBECF91213B1
:10433B00C5900908E0FAA3E0D283F5A0C280D28031
:10434B00EAF5A0C280D280C283900B5EE0F8A3E0B6
:10435B00F9900908E8F0A3E9F0850C82850D83E05C
:10436B0024F8F50AEEFAEFFBA90A1213C590090817
:10437B00E0FAA3E0D283F5A0C280D280EAF5A0C216
:10438B0080D280C283850882850983E50AF0EE24FA
:10439B00010EEF3400FF850C82850D83A385820C03
:1043AB0085830D850882850983A38582088583090A
:1043BB00850E82850F83A385820E85830FC3EE94B2
:1043CB008FEF9401500302429B02176C74F1120E93
:1043DB000074FA120D96D2A8C2909008F9E0A2E4EC
:1043EB0050F8E0C2E4F0C2A8D290123DF17402651D
:1043FB002170057522018007E52270030246E97ED4
:10440B00007F007404120DE17429F0A37405F0749D
:10441B0002120DE1741DF0A37407F0750CA5750D58
:10442B0001750835750903A82274C528FA7404347C
:10443B0000FB851082851183EAF0A3EBF074B92899
:10444B00F50E74063400F50F75A60075A0FFC29724
:10445B0085A00A743B250AF58274853400F583E444
:10446B0093C0E07404120DE1E0F8A3E0F5838882B9
:10447B00D0E0F0D297C29585A00A743B250AF5824D
:10448B0074853400F583E493C0E07402120DE1E00F
:10449B00F8A3E0F5838882D0E0F0D29575A6FF856E
:1044AB000C82850D83E0FC74786C600874C86E70A8
:1044BB0001EF700B90090874EFF0A3747B8052EC42
:1044CB0075F00584E5F07012EEF8EFF97A197B00C0
:1044DB00120D1A8B0BEA450B60DAEC2405F8E43469
:1044EB0000F97A197B00120D128B0BEA450B701237
:1044FB00EEF8EFF97A057B00120D1A8B0BEA450BE0
:10450B0060B2900902E0F8A3E0F9900908E8F0A383
:10451B00E9F0EEFAEFFBECF91213C5900908E0FA9B
:10452B00A3E0D283F5A0C280D280EAF5A0C280D2EC
:10453B0080C283850882850983E0FC74786C6008EF
:10454B0074C86E7001EF700B90090874EFF0A374D0
:10455B007B8052EC75F00584E5F07012EEF8EFF904
:10456B007A197B00120D1A8B0BEA450B60DAEC24DF
:10457B0005F8E43400F97A197B00120D128B0BEA63
:10458B00450B7012EEF8EFF97A057B00120D1A8BC2
:10459B000BEA450B60B2900902E0F8A3E0F9900931
:1045AB0008E8F0A3E9F0EEFAEFFBECF91213C59073
:1045BB000908E0FAA3E0D283F5A0C280D280EAF525
:1045CB00A0C280D280C283900B5CE0F8A3E0F9908C
:1045DB000908E8F0A3E9F0851082851183E0F8A3C0
:1045EB00E0F5838882E0246AF50AEEFAEFFBA90A6C
:1045FB001213C5900908E0FAA3E0D283F5A0C2809C
:10460B00D280EAF5A0C280D280C283850C82850D50
:10461B0083E50AF0900B5EE0F8A3E0F9900908E857
:10462B00F0A3E9F0850E82850F83E02406F50AEEF0
:10463B00FAEFFBA90A1213C5900908E0FAA3E0D21E
:10464B0083F5A0C280D280EAF5A0C280D280C2835B
:10465B00850882850983E50AF0EE24010EEF34000C
:10466B00FF850E82850F83A385820E85830F8510B0
:10467B0082851183E02401F8A3E03400F9851082D0
:10468B00851183E8F0A3E9F0850882850983A3856A
:10469B008208858309850C82850D83A385820C8511
:1046AB00830D7402120DE1E02401F8A3E03400F94C
:1046BB007402120DE1E8F0A3E9F07404120DE1E0CD
:1046CB002401F8A3E03400F97404120DE1E8F0A31F
:1046DB00E9F0C3EE948FEF94015003024453C2965A
:1046EB00D296740602364174F3120E00D2A8C29011
:1046FB009008F9E0A2E450F8E0C2E4F0C2A8123F3F
:10470B009E7402652170057522018007E5227003F6
:10471B0002489775A60075A0FF7E007F0078297967
:10472B0005C29785A008743B2508F5827486340072
:10473B00F583E49388828983F0D297C29585A0088C
:10474B00743B2508F58274863400F583E4938882E4
:10475B008983A3F0D295EE24020E0EEF3400FFE80E
:10476B0024020808E93400F9C3EE948EEF9401405B
:10477B00B075A6FF7E007F007508A575090185221F
:10478B000A74C5250AF50C74043400F50D850882EE
:10479B00850983E0FC74786C600874C86E7001EF57
:1047AB00700B90090874EFF0A3747B8052EC75F0DA
:1047BB000584E5F07012EEF8EFF97A197B00120D13
:1047CB001A8B0BEA450B60DAEC2405F8E43400F99C
:1047DB007A197B00120D128B0BEA450B7012EEF857
:1047EB00EFF97A057B00120D1A8B0BEA450B60B2C1
:1047FB00900902E0F8A3E0F9900908E8F0A3E9F0CA
:10480B00EEFAEFFBECF91213C5900908E0FAA3E0FE
:10481B00D283F5A0C280D280EAF5A0C280D280C23A
:10482B008390090874FFF0A3F0850C82850D83E05B
:10483B0024F8F50AEEFAEFFBA90A1213C590090842
:10484B00E0FAA3E0D283F5A0C280D280EAF5A0C241
:10485B0080D280C283850882850983E50AF0EE2425
:10486B00010EEF3400FF850C82850D83A385820C2E
:10487B0085830D850882850983A385820885830935
:10488B00C3EE948FEF94015003024798C296D296D1
:10489B007F06020E6674F5120E00900908E0F5080B
:1048AB00A3E0F509900908E4F0A374F8F09008FD73
:1048BB00E0F8E0A2E6E43344FEF4F9E8A2E7E433DF
:1048CB0044FEF49008F2F8E028C399F0F4700474F5
:1048DB00088007E0C394094002E4F09008B9E0F8BF
:1048EB009008F2E0686003121A68900B60E0F8A37E
:1048FB00E0F9900906E8F0A3E9F090090474FFF0E1
:10490B00A3F09008F2E06033147003024AAA14700B
:10491B0003024B15147003024B80147003024BF807
:10492B00147003024C6C147003024CD0147003020D
:10493B004FAB14700302501302507F9008FDE0A29E
:10494B00E49008F15003024AA2E0F8740128F0E861
:10495B00C39410500302507F900AF1E09008B7F017
:10496B00900AF2E09008B8F09008FAE0D2E4F01266
:10497B002848900B5CE0F8A3E0F990090CE8F0A351
:10498B00E9F0900B5EE0F8A3E0F990090EE8F0A3D4
:10499B00E9F0900902E0F8A3E0F9900910E8F0A320
:1049AB00E9F0800AD2ADE0A2E55003122905900888
:1049BB00FAE0A2E440EE9008B7E0900AF1F090081C
:1049CB00B8E0900AF2F0900AF1E0FEC3940590086B
:1049DB00EBE04004C2E08002D2E0F09008FCE0542F
:1049EB00EDF09008EBE09008E7F0795D121E8990EE
:1049FB0008FCE054EDF0EEC333F8E433F974B1285E
:104A0B00F582748939F583E4939008E7F0794812BD
:104A1B001E89900AF2E0FEC394059008EBE0400477
:104A2B00C2E18002D2E1F09008FCE054EDF0900876
:104A3B00EBE09008E7F0795D121E899008FCE054DA
:104A4B00EDF0EEC333F8E433F974B128F5827489D1
:104A5B0039F583E4939008E7F07949121E899008A1
:104A6B00F1E4F0900902E0F8A3E0F9900906E8F010
:104A7B00A3E9F0750A8F750B01780A120EA67CDE7E
:104A8B007A007B0079141214EC7402120DAC12191B
:104A9B008E121A6802507FE4F012509B02507F90E6
:104AAB0008FBE0C2E0F07E127F007C0D7D00EEFA89
:104ABB00EFFB79021219017C0D7D00EE2401FAEF58
:104ACB003400FB7902121901EE240AFEEF3400FFC9
:104ADB0074586E7001EF70D27582F775830A7E146D
:104AEB007F008012EEFAEFFB79021215DBEE240A3F
:104AFB00FEEF3400FFA3E0FC743F6C70E7900906F7
:104B0B00E4F0A3F0125A8D02507F9008FBE0C2E054
:104B1B00F07E587F007C0D7D00EEFAEFFB790212E0
:104B2B0019017C0D7D00EE2401FAEF3400FB7902B4
:104B3B00121901EE240AFEEF3400FF74BC6E7001F3
:104B4B00EF70D275820175830B7E5A7F008012EE57
:104B5B00FAEFFB79021215DBEE240AFEEF3400FFAD
:104B6B00A3E0FC743F6C70E7900906E4F0A3F0122D
:104B7B0056B202507F9008FBE0C2E0F07EBC7F0093
:104B8B007C0D7D00EEFAEFFB79021219017C0D7D95
:104B9B0000EE2401FAEF3400FB7902121901EE2426
:104BAB000AFEEF3400FF74206E700374016F70D037
:104BBB00900B5CE0F8A3E0F9900904E8F0A3E9F0AE
:104BCB0075820B75830B7EBE7F008012EEFAEFFBB6
:104BDB0079021215DBEE240AFEEF3400FFA3E0FC92
:104BEB00743F6C70E77900125CD002507F9008FB29
:104BFB00E0C2E0F07E207F017C0D7D00EEFAEFFB42
:104C0B0079021219017C0D7D00EE2401FAEF3400BC
:104C1B00FB7902121901EE240AFEEF3400FF7484B3
:104C2B006E700374016F70D0900B5EE0F8A3E0F927
:104C3B00900904E8F0A3E9F075821575830B7E22C9
:104C4B007F018012EEFAEFFB79021215DBEE240ADC
:104C5B00FEEF3400FFA3E0FC743F6C70E77901803A
:104C6B00869008FBE0C2E0F07E127F007C0D7D0099
:104C7B00EEFAEFFB79E11219017C0D7D00EE2401B8
:104C8B00FAEF3400FB79E1121901EE240AFEEF343E
:104C9B0000FF74586E7001EF70D275821F75830B15
:104CAB007E147F008012EEFAEFFB79E11215DBEE3A
:104CBB00240AFEEF3400FFA3E0FC743F6C70E71294
:104CCB00592E02507F9008FBE0C2E0F07E587F0027
:104CDB007C0D7D00EEFAEFFB79E11219017C0D7D65
:104CEB0000EE2401FAEF3400FB79E1121901EE24F6
:104CFB000AFEEF3400FF74946E7001EF70D2758270
:104D0B002975830B7E5A7F008012EEFAEFFB79E157
:104D1B001215DBEE240AFEEF3400FFA3E0FC743F18
:104D2B006C70E79008F9E0A2E74003024E1F900871
:104D3B00FDE0A2E55003024F0A9008F9E0C2E7F04C
:104D4B00900902E0F8A3E0F9900906E8F0A3E9F076
:104D5B00750A8F750B01780A120EA67CDE7A007B22
:104D6B000079141214EC7402120DAC12198E7EAD74
:104D7B007F089008F7E0F8A3E0F9E875F006A4F8CF
:104D8B00AAF075F006E9A42AF974E328FC748739B4
:104D9B00FDECF8EDF97AF77B0A88828983E493F5C9
:104DAB000A8E828F83F0EA240BF582EB3400F583B5
:104DBB00E50AF08A828B83A3AA82AB8388828983DC
:104DCB00A3A882A9838E828F83A3AE82AF83EAB41A
:104DDB00FC03EB640A70C28C828D83A3A3A3A3A3F1
:104DEB00E4939008B2F0900906E4F0A3F07582AD5D
:104DFB007583087E64FFE0FC743F6C7003024F0AFE
:104E0B00EEFAEFFB79021215DBEE240AFEEF34000B
:104E1B00FFA380E2E0A2E75003024F0A9008FDE0F7
:104E2B00A2E45003024F0A9008F9E0D2E7F0900990
:104E3B0002E0F8A3E0F9900906E8F0A3E9F0750A9F
:104E4B008F750B01780A120EA67CDE7A007B007937
:104E5B00141214EC7402120DAC12198E7EAD7F0875
:104E6B009008F7E0F8A3E0F9E875F006A4F8AAF0CB
:104E7B0075F006E9A42AF9743B28FC748739FDEC1C
:104E8B00F8EDF97AF77B0A88828983E493F50A8E29
:104E9B00828F83F0EA240BF582EB3400F583E50A6D
:104EAB00F08A828B83A3AA82AB8388828983A3A88F
:104EBB0082A9838E828F83A3AE82AF83EAB4FC0375
:104ECB00EB640A70C28C828D83A3A3A3A3A3E49388
:104EDB009008B2F0900906E4F0A3F07582AD7583EB
:104EEB00087E64FF8012EEFAEFFB79021215DBEEFF
:104EFB00240AFEEF3400FFA3E0FC743F6C70E790D4
:104F0B000906E4F0A374F8F09008F9E0A2E7503436
:104F1B00C2B075128090090474E0F0A37407F075A9
:104F2B0082DA75830A7E647F00E0FC743F6C6066F6
:104F3B00EEFAEFFB79E11215DBEE240AFEEF3400FB
:104F4B00FFA380E59008FAE0F8E0F9E8A2E0500A48
:104F5B00E9A2E15005751240800DE0A2E04005E0AA
:104F6B00A2E15003751280D2B090090474FFF0A334
:104F7B00F07582DA75830A7E647F008012EEFAEF99
:104F8B00FB79E11215DBEE240AFEEF3400FFA3E000
:104F9B00FC743F6C70E7900906E4F0A3F002507FBD
:104FAB009008FBE0C2E0F07E947F007C0D7D00EE6C
:104FBB00FAEFFB79E11219017C0D7D00EE2401FA69
:104FCB00EF3400FB79E1121901EE240AFEEF3400F5
:104FDB00FF74E46E7001EF70D275823375830B7EB4
:104FEB00967F008012EEFAEFFB79E11215DBEE24CF
:104FFB000AFEEF3400FFA3E0FC743F6C70E79009EE
:10500B0006E4F0A3F0F980699008FBE0C2E0F07EC3
:10501B00E47F007C0D7D00EEFAEFFB79E1121901C4
:10502B007C0D7D00EE2401FAEF3400FB79E11219BF
:10503B0001EE240AFEEF3400FF74346E700374012A
:10504B006F70D075823D75830B7EE67F008012EE0C
:10505B00FAEFFB79E11215DBEE240AFEEF3400FFC9
:10506B00A3E0FC743F6C70E7900906E4F0A3F079C1
:10507B0001125B98900906E4F0A3F0900908E5088B
:10508B00F0A3E509F09008F2E09008B9F00215746E
:10509B0074F7120E009008F9E0A2E750030256AF26
:1050AB009008FDE0A2E05005E0A2E1402E9009023D
:1050BB00E0F8A3E0F9900906E8F0A3E9F075088F92
:1050CB007509017808120EA67CDE7A007B00791434
:1050DB001214EC7402120DAC12198E9008FAE0F84F
:1050EB00E0F9E8A2E05027E9A2E150229008FDE0A8
:1050FB00A2E0400A9008FAE0C2E0F0751280900836
:10510B00FDE0A2E1406F9008FAE0C2E18063E0A20B
:10511B00E050269008FDE0A2E0400A9008FAE0C2B9
:10512B00E0F07512809008FDE0A2E140489008FA8B
:10513B00E0D2E1F0751240803CE0A2E19008FDE086
:10514B005018A2E0400A9008FAE0D2E0F075124045
:10515B009008FDE0A2E1401D80ACA2E04008900861
:10516B00FAE0D2E0800BE0A2E1400A9008FAE0D22C
:10517B00E1F07512809008FAE0F8E0F9E8A2E0405F
:10518B00030253B1E9A2E140030253B1900902E0DB
:10519B00F8A3E0F9900906E8F0A3E9F0900B5CE0C6
:1051AB00F8A3E0F9900904E8F0A3E9F07A007CADEC
:1051BB007D0878F7790A8A08900AF1E075F005A462
:1051CB00FEAFF074612EFE74893FFFEE2508F58269
:1051DB00EF3400F583E493FB8C828D83F0EAC39468
:1051EB0004500CE82415F582E93400F583EBF00A42
:1051FB0088828983A3A882A9838C828D83A3AC82A6
:10520B00AD83EAC3940540AE7582AD7583087EC845
:10521B007F008012EEFAEFFB79021215DBEE240A07
:10522B00FEEF3400FFA3E0FC743F6C70E7900902C3
:10523B00E0F8A3E0F9900906E8F0A3E9F0900B5E23
:10524B00E0F8A3E0F9900904E8F0A3E9F07A007C18
:10525B00AD7D0878F7790A8A08900AF2E075F005B7
:10526B00A4FEAFF074612EFE74893FFFEE2508F5A6
:10527B0082EF3400F583E493FB8C828D83F0EAC3D9
:10528B009404500CE8241FF582E93400F583EBF00D
:10529B000A88828983A3A882A9838C828D83A3AC7D
:1052AB0082AD83EAC3940540AE7582AD7583087EEB
:1052BB002C7F018012EEFAEFFB79021215DBEE2444
:1052CB000AFEEF3400FFA3E0FC743F6C70E785121D
:1052DB00087509007808120EA67CDF7D0A7AE97B37
:1052EB000A1288B37402120DAC900AEB7420F09082
:1052FB0008FAE0A2E65007900AEC747B800AE0A261
:10530B00E64006900AEC747DF0900AED7420F0A351
:10531B00743FF07AF87B0A78E9790A88828983E00E
:10532B008A828B83F088828983A3A882A9838A824D
:10533B008B83A3AA82AB83E8B4EF03E9640A70DB27
:10534B00900902E0F8A3E0F9900906E8F0A3E9F070
:10535B0074026521700990090474FFF0A3801EE5A7
:10536B00217005900B5C8009740165217010900B06
:10537B005EE0F8A3E0F9900904E8F0A3E9F0758288
:10538B00E975830A7E1E7F00E0FC743F6C7003029C
:10539B0056AFEEFAEFFB79021215DBEE240AFEEFA5
:1053AB003400FFA380E2E0A2E0400302552C9009F9
:1053BB0002E0F8A3E0F9900906E8F0A3E9F0900BFE
:1053CB005CE0F8A3E0F9900904E8F0A3E9F07A00B7
:1053DB007CAD7D0878F7790A8A08900AF1E075F0C0
:1053EB0005A4FEAFF074892EFE74893FFFEE2508ED
:1053FB00F582EF3400F583E493FB8C828D83F0EA26
:10540B00C39404500CE82415F582E93400F583EBC2
:10541B00F00A88828983A3A882A9838C828D83A3B7
:10542B00AC82AD83EAC3940540AE7582AD7583083B
:10543B007EC87F008012EEFAEFFB79021215DBEECD
:10544B00240AFEEF3400FFA3E0FC743F6C70E78589
:10545B0012087509007808120EA67CDF7D0A7AE91E
:10546B007B0A1288B37402120DAC9008FAE0A2E624
:10547B005007900AEC747B800AE0A2E64006900A83
:10548B00EC747DF0900AED7420F0A3743FF07AF881
:10549B007B0A78E9790A88828983E08A828B83F098
:1054AB0088828983A3A882A9838A828B83A3AA82F9
:1054BB00AB83E8B4EF03E9640A70DB900902E0F810
:1054CB00A3E0F9900906E8F0A3E9F07402652170F6
:1054DB000990090474FFF0A3801EE5217005900B61
:1054EB005C8009740165217010900B5EE0F8A3E0FD
:1054FB00F9900904E8F0A3E9F07582E975830A7E57
:10550B001E7F00E0FC743F6C70030256A7EEFAEFAF
:10551B00FB79021215DBEE240AFEEF3400FFA380A9
:10552B00E2E0A2E140030256AF900902E0F8A3E0EB
:10553B00F9900906E8F0A3E9F0900B5EE0F8A3E020
:10554B00F9900904E8F0A3E9F07A007CAD7D0878C6
:10555B00F7790A8A08900AF2E075F005A4FEAFF01D
:10556B0074892EFE74893FFFEE2508F582EF340017
:10557B00F583E493FB8C828D83F0EAC39404500C87
:10558B00E8241FF582E93400F583EBF00A88828961
:10559B0083A3A882A9838C828D83A3AC82AD83EA7B
:1055AB00C3940540AE7582AD7583087E2C7F018058
:1055BB0012EEFAEFFB79021215DBEE240AFEEF3442
:1055CB0000FFA3E0FC743F6C70E7751280750880D8
:1055DB007509007808120EA67CDF7D0A7AE97B0A32
:1055EB001288B37402120DAC9008FAE0A2E65007D1
:1055FB00900AEC747B800AE0A2E64006900AEC74F9
:10560B007DF0900AED7420F0A3743FF07AF87B0ADA
:10561B0078E9790A88828983E08A828B83F0888291
:10562B008983A3A882A9838A828B83A3AA82AB8353
:10563B00E8B4EF03E9640A70DB900902E0F8A3E039
:10564B00F9900906E8F0A3E9F0740265217009905E
:10565B00090474FFF0A3801EE5217005900B5C809C
:10566B0009740165217010900B5EE0F8A3E0F990CE
:10567B000904E8F0A3E9F07582E975830A7E1E7FC1
:10568B00008012EEFAEFFB79021215DBEE240AFE14
:10569B00EF3400FFA3E0FC743F6C70E790090474D7
:1056AB00FFF0A3F002355974F7120E009009047441
:1056BB00FFF0A3F09008FDE0A2E4500302575390D3
:1056CB0008FEE0A2E09008F75025E02401F0A3E0EB
:1056DB003400F09008F7C3E0941CA3E09400A2D22E
:1056EB0065D033403C9008F7741BF0A3E48031C3C2
:1056FB00E09418A3E09400A2D265D0339008F7E0B1
:10570B0040102401F0A3E03400F09008FEE0D2E05A
:10571B00800E2401F0A3E03400F09008FEE0C2E01C
:10572B00F09008FEE0C2E1F0E0A2E150549008F5E1
:10573B007418F09008F67440F09008E77402F0903B
:10574B0008FEE0D2E202583AE0A2E5402B9008F7BF
:10575B00E024FFF0F8A3E034FFF0F9C3E89401E98B
:10576B009400A2D265D03350B89008F7E4F0A3F0C0
:10577B009008FEE0D2E180AF900906E4F0A3025955
:10578B002AE0A2E050559008F7E0F508A3E0F509F0
:10579B007808120EE6180003DF57AD57C057C757EE
:1057AB00D3579008F57418F09008F6E4F09008FEC3
:1057BB00E0C2E0801E9008F5741880119008F57413
:1057CB0019F09008F6E4800B9008F57419F0900826
:1057DB00F67480F09008E774028054E0A2E2500760
:1057EB009008F5741880DA9008F7E0F8A3E0F9E870
:1057FB00C333F8E933F9742928F582748939F583B1
:10580B00E493C0E0740193F583D082AA82AB838AC0
:10581B00088B0974027808120D73E5089008F5F0EF
:10582B00EAC4333354C09008F6F09008E77401F0E3
:10583B007E007508AD7509089008F7E0F8A3E0F94C
:10584B00E875F006A4F8AAF075F006E9A42AF97435
:10585B003B28FA748739FB74E328F8748739F97C91
:10586B00F77D0A9008F9E0A2E750068A828B8380C5
:10587B000488828983E493850882850983F0EEC3CB
:10588B0094055010E0C0E0EC240BF582ED3400F5EC
:10589B0083D0E0F00E8C828D83A3AC82AD838882A3
:1058AB008983A3A882A9838A828B83A3AA82AB83D1
:1058BB00850882850983A3858208858309EEC394B5
:1058CB000640A0900906E4F0A374F8F07582AD755C
:1058DB0083087E647F008012EEFAEFFB79021215CB
:1058EB00DBEE240AFEEF3400FFA3E0FC743F6C7088
:1058FB00E7900906E4F0A3F09008F5E09008E8F0D3
:10590B009008F6E09008E9F09008F9E0C2E3F0E0C7
:10591B00D2E2F09008FCE0D2E1F0900AF57459F075
:10592B0002355974F7120E009008FDE0A2E04049D1
:10593B00E5216015900B5CE0F8A3E0F9900904E811
:10594B00F0A3E9F0752100800B7521029009047416
:10595B00FFF0A3F07582E375830A7E1E7F00E0FCE7
:10596B00743F6C6064EEFAEFFB79E11215DBEE2409
:10597B000AFEEF3400FFA380E5E0A2E1404B740187
:10598B0065216015900B5EE0F8A3E0F9900904E83F
:10599B00F0A3E9F0752101800B75210290090474C5
:1059AB00FFF0A3F07582E375830A7E1E7F008012E1
:1059BB00EEFAEFFB79E11215DBEE240AFEEF340071
:1059CB00FFA3E0FC743F6C70E78512087509007843
:1059DB0008120EA67CDF7D0A7AE97B0A1288B37463
:1059EB0002120DACE512C394645006900AEB7420BE
:1059FB00F09008FAE0A2E65007900AEC747B800A5C
:105A0B00E0A2E64006900AEC747DF0900AED74205B
:105A1B00F0A3743FF07AF87B0A78E9790A888289D7
:105A2B0083E08A828B83F088828983A3A882A983EF
:105A3B008A828B83A3AA82AB83E8B4EF03E9640A5F
:105A4B0070DB900902E0F8A3E0F9900906E8F0A3F7
:105A5B00E9F07582E975830A7E1E7F008012EEFAEB
:105A6B00EFFB79021215DBEE240AFEEF3400FFA3E5
:105A7B00E0FC743F6C70E790090474FFF0A3F00234
:105A8B00355974F7120E009008FDE0A2E4400405AE
:105A9B00128031E0A2E5400415128028E0A2E0401C
:105AAB000E9008FAE0D2E6F0900AEC747B8014E0DA
:105ABB00A2E15003025B959008FAE0C2E6F0900A6F
:105ACB00EC747DF08512087509007808120EA67C1F
:105ADB00DF7D0A7AE97B0A1288B37402120DACE5FA
:105AEB0012C394645006900AEB7420F09008FAE00D
:105AFB00A2E65007900AEC747B800AE0A2E640060F
:105B0B00900AEC747DF0900AED7420F0A3743FF0D2
:105B1B007AF87B0A78E9790A88828983E08A828B12
:105B2B0083F088828983A3A882A9838A828B83A32B
:105B3B00AA82AB83E8B4EF03E9640A70DB90090433
:105B4B0074FFF0A3F0900B60E0F8A3E0F990090666
:105B5B00E8F0A3E9F07582E975830A7E1E7F008069
:105B6B0012EEFAEFFB79021215DBEE240AFEEF348C
:105B7B0000FFA3E0FC743F6C70E7900902E0F8A310
:105B8B00E0F9900906E8F0A3E9F002355974F41234
:105B9B000E00E9FF750800A2A8E433F509A2ACE4F6
:105BAB0033F50AA2ADE433F50BC2A8C2ACC2AD907B
:105BBB0008FDE0A2E04050EF704D7827A6EA08748C
:105BCB002E6870F87523EED2AD900B62E060FAC2CE
:105BDB00AD750C047E279008E7E4F0E50C9008E81F
:105BEB00F0EEF8E69008E9F09008FCE0C2E4F0D2A1
:105BFB00E1F07950121E89D2ADC2AD050C0EE50C49
:105C0B00C3940C505780CFE0A2E1407B74016F70BE
:105C1B0076782FA6FC0874366870F87523EED2AD33
:105C2B00900B62E060FAC2AD750C0C7E2F9008E70A
:105C3B00E4F0E50C9008E8F0EEF8E69008E9F09057
:105C4B0008FCE0C2E4F0D2E1F07950121E89D2AD2B
:105C5B00C2AD050C0EE50CC3941440D1D2AD900827
:105C6B00E7E4F09008E8F0E5239008E9F09008FCF1
:105C7B00E0C2E4F0D2E1F07950121E89EF701CE51E
:105C8B000825EAF5EA801AE0A2E4400575080180D0
:105C9B00EBE0A2E5400B7508FF80E1E50825FCF57C
:105CAB00FCE5A854FE4509F5A8E50AC4F8E5A85497
:105CBB00EF48F5A8E50BC43354E0F8E5A854DF48EA
:105CCB00F5A80240C074F6120E008908E9600302C1
:105CDB005DFF9008FDE0A2E4400F900AF1E004F0B4
:105CEB00C39408401974078014E0A2E55003025FC7
:105CFB0039900AF1E014F0C394C94002E4F075093D
:105D0B00007AAD7B0878F7790A850982AC82900816
:105D1B00FAE0A2E1900AF1E075F005500FA4FE85C0
:105D2B00F00AAF0A74612EFE7489800DA4FE85F013
:105D3B000AAF0A74892EFE74893FFFEE2CF582EFB1
:105D4B003400F583E4938A828B83F0ECC394045084
:105D5B0010E0C0E0E82415F582E93400F583D0E0CB
:105D6B00F0050988828983A3A882A9838A828B8301
:105D7B00A3AA82AB83E509C39405408D7582AD75EB
:105D8B0083087EC87F008012EEFAEFFB79021215B2
:105D9B00DBEE240AFEEF3400FFA3E0FC743F6C70D3
:105DAB00E7900AF1E02427F8E6F5EAE0FEC3940554
:105DBB009008EBE04004C2E08002D2E0F09008FCD7
:105DCB00E054EDF09008EBE09008E7F0795D121EDF
:105DDB00899008FCE054EDF0EEC333F8E433F9742A
:105DEB00B128F582748939F583E4939008E7F0794B
:105DFB0048025F27740165086003025F2A9008FD63
:105E0B00E0A2E4400F900AF2E004F0C394084019BA
:105E1B0074078014E0A2E55003025F39900AF2E0A8
:105E2B0014F0C394C94002E4F07509007AAD7B0805
:105E3B0078F7790A850982AC829008FAE0A2E090A3
:105E4B000AF2E075F005500FA4FE85F00AAF0A7454
:105E5B00612EFE7489800DA4FE85F00AAF0A748949
:105E6B002EFE74893FFFEE2CF582EF3400F583E4B0
:105E7B00938A828B83F0ECC394045010E0C0E0E86B
:105E8B00241FF582E93400F583D0E0F00509888200
:105E9B008983A3A882A9838A828B83A3AA82AB83DB
:105EAB00E509C39405408D7582AD7583087E2C7F03
:105EBB00018012EEFAEFFB79021215DBEE240AFEDB
:105ECB00EF3400FFA3E0FC743F6C70E7900AF2E044
:105EDB00242EF8E6F5FCE0FEC394059008EBE040B9
:105EEB0004C2E18002D2E1F09008FCE054EDF090A6
:105EFB0008EBE09008E7F0795D121E899008FCE052
:105F0B0054EDF0EEC333F8E433F974B128F5827431
:105F1B008939F583E4939008E7F07949121E89904B
:105F2B000906E4F0A3F090090474FFF0A3F0021942
:105F3B008974F1120E0074FD120D967402120DE1AC
:105F4B00E9F08A088B098C0A8D0B7414120DE1E0B1
:105F5B00FEA3E0FF851082851183E4F0A3F08E820F
:105F6B008F83A3AA82AB83900B99780C120C757854
:105F7B0008790C1204FA70188E828F83746912647C
:105F8B001B746EF0A37466F0A30A0AAB830263B6AC
:105F9B00780879081204FA60118E828F83746E125E
:105FAB00641B7461F0A3746E80DD900B9D780C12F2
:105FBB000C757808790C1205265003026066900B5D
:105FCB0065780C120C757808790C1204FA600302D0
:105FDB0060BA7416120DE1E070030260FC8510824A
:105FEB00851183C082C0837412120DE1126E59D0D9
:105FFB0083D0821263F4502C851082851183C3E009
:10600B0094FCA3E094FFA2D265D033401774021224
:10601B000DE1E4126F2DF97412120DE1C3E098F04B
:10602B00A3E099F07412120DE11264117417120DA2
:10603B00E1E070030260F97416120DE1E40260FBFB
:10604B00900BA1780C120C757808790C12097D85D0
:10605B001082851183E0240A126F6A900BA5780CCD
:10606B00120C757808790C12052640D4900BA97880
:10607B000C120C757808790C1205264003025FDDB3
:10608B00900BA9780C120C757808790C12097D12FB
:10609B006F6180D8900BA1780C120C757808790C75
:1060AB001205C1851082851183E024F612641490C9
:1060BB000BAD780C120C757808790C12057540D461
:1060CB00900B9D780C120C757808790C12057540A5
:1060DB0003025FDD900BA9780C120C757808790C14
:1060EB001205C185108285118312641180D274014F
:1060FB00F07402120DE1E060077A007B0002620887
:10610B00126400507D8E828F837430F0EAFEEBFFB9
:10611B007412120DE1E0FCA3E0FDEC4D7008741756
:10612B00120DE1E0600B8E828F83742EF0A30EAF05
:10613B00837A007B0080118E828F83743012643CD3
:10614B007412120DE1126411EA24FF1AEB34FFFBF7
:10615B008510828511831263E8500B7412120DE1C6
:10616B00126E5D4970D185108285118374FFC39CBB
:10617B00F874FF9DF91263F450030262D67A0102A0
:10618B006106851082851183126E59C3E498FAE477
:10619B0099FB806985080C85090D850A0E850B0F07
:1061AB00780C12040FAC0CE50D3395E0F50EF50FE2
:1061BB00780C1203977808790C120741900BA97889
:1061CB000C120C757808790C1205C1EC126436EAC6
:1061DB00F8EBF9E824010AE93400FBE849701E7476
:1061EB0012120DE1126E5D4970087417120DE1E089
:1061FB00600B8E828F83742EF0A30EAF83741212FA
:10620B000DE11263E8508D900BB1780C120C757880
:10621B0008790C12052640030262D67C01EE24FF9E
:10622B00F8EF34FFF97414120DE1E0F508A3E0F573
:10623B000988828983E0642E6010E02CF0643A7048
:10624B00077430F07C0180027C00E8FAE9FBEA2459
:10625B00FF18EB34FFF9C3E5089AE5099B40D2EC34
:10626B00A2E050677402120DE1E06036EEF8EF80A9
:10627B000A1263D3E824FF18E934FFF9C3E5089841
:10628B00E5099950181263C0E0642E70E4E824FE0F
:10629B00F582E934FFF5831263CDF980D7126F6174
:1062AB00801E8E828F83A3AE82AF83EEF8EF8006C3
:1062BB001263C01263CDF9C3E50898E5099940F064
:1062CB007414120DE1126E787431F07416120DE124
:1062DB00E07005801A1EAF83EE24FFF582EF34FFCA
:1062EB00F583E0643060EEE0642E70031EAF8374C0
:1062FB0002120DE1E070030263B2126438A3A983AA
:10630B001264008E828F835014742DF00EE9FF857A
:10631B001082851183126EA11264298006742BF0F2
:10632B000EE9FF7C007D00EE240AFEEF3400FFEC4B
:10633B0024010CED3400FD1263DA120D12EA126423
:10634B00361263DA120D121264434970E2C3EC94F5
:10635B0002ED126E0A40D8ECFAEDFBC3E49CF8E4B4
:10636B009DF9EE28F582EF39F583E0C0E0C3E49A9E
:10637B00F8E49BF9EE28F8EF39F9E82CF8E93DF948
:10638B00E824F5F582E934FFF583D0E0F0EC24FF47
:10639B001CED34FFFDC3EC9401ED126E0A50BCEE04
:1063AB0024F6FEEF34FFFFEEFAEFFB7403120DAC95
:1063BB007F08020E66E824FFFAE934FFFB8A828B22
:1063CB0083221263D318EB22E088828983F0228523
:1063DB001082851183126EAE7A0A7B0022C3E09A7B
:1063EB00A3E09BA2D265D03322C3E098A3E099A28D
:1063FB00D265D03322851082851183C3A3E094002C
:10640B00A2D265D03322E024FFF0A3E034FFF022C8
:10641B00F0EAFEEBFF8E828F8322A3E03400F98536
:10642B001082851183E8F0A3E9F02224308E828F4D
:10643B0083F0A3AE82AF8322851082851183126411
:10644B004D22E8F0A3E9F0851082851183E02274D8
:10645B00F1120E0074B0120D968510828511831205
:10646B006F137418120DE1ECF0A3EDF0740F120D15
:10647B00E1E4F0A38022745F120DE1126E49740403
:10648B00120DE1E0F97418120DE1126E78120DEB9A
:10649B00740F120DE1126E12F0126E8CFA126F4C19
:1064AB00120DE1EAF074256A6010E070C9740F12E6
:1064BB000DE1126E4974500263B8126E8C64257034
:1064CB0019851082851183E0240108126425745FFD
:1064DB00120DE1126E49792580AB740E120DE1E4B9
:1064EB00F0740D120DE1E4F0740C120DE1E4F07494
:1064FB0005120DE1E4F0741E120DE1A882A983745C
:10650B0002120DE180157405120DE1E070077405A0
:10651B00120DE1EAF0851082851183126449126E27
:10652B0040126ED3FA24E060DD24FD601724F8607E
:10653B00DD24FE600624FD600F8011740C120DE14A
:10654B00E00480D0740D80F5740E80F1126ED3646C
:10655B002A705B7461120DE1126EDEFB8A828B83F3
:10656B00E0FCA3E0FD740A120DE1ECF0A3EDF0EA00
:10657B0024020A0AEB3400FB7461120DE1126F0B5B
:10658B00740A120DE1126406501F740A120DE11207
:10659B006E49C3E49AFAE49BFB740A120DE1126F85
:1065AB0013740C120DE1E004F012642A804A740A91
:1065BB00120DE1E4F0A3802D740A120DE1126E5D51
:1065CB0075F00AA4F8AAF075F00AE9A42AF9E5080F
:1065DB0028F8E439F9E824D0F8E934FFF9740A1201
:1065EB000DE1126F71126F2DF5838882E0F508743F
:1065FB00D02508C3940A40C0740C120DE1E060076B
:10660B00740E120DE1E4F0126E8C642E60030266C0
:10661B00A5851082851183E0240108A3E03400F9DD
:10662B00126443126E7DE0642A702C7461120DE1CA
:10663B00126E92F8A3E0F988828983E0FEA3E0FF53
:10664B00E824020808E93400F97461120DE1126EB6
:10665B00C6126F71F080477E007F00851082851116
:10666B0083126E9B74D02508C3940A5031EE75F0DB
:10667B000AA4FEA8F075F00AEFA428FFE5082EF88F
:10668B00E43FF9E824D0FEE934FFFF851082851141
:10669B0083E02401F812642580C17EFF7FFF7A001E
:1066AB00851082851183126E3B851082851183E0E4
:1066BB00FBA3E0F5838B82E024B4600824E460053F
:1066CB0024FC70040A12642A126E8CFB126F4C129B
:1066DB000DE1EBF07003026CB024BB7003026B7620
:1066EB0024FE7003026B5824EF70030268A224F59A
:1066FB0070030267A7147003026947147003026BDF
:10670B0076147003026B74147003026B5824FE70C2
:10671B000302694724FB602414700302689214700F
:10672B00030268A224FD70030267E024FE700302DB
:10673B0068A224FD70030268A2026CBC7461120D86
:10674B00E1126F05120DE1126430EAA2E0740F50F2
:10675B0033120DE1E0FCA3E0FD3395E0FE7406126D
:10676B000DE1126EE6ECF0A3EDF0A3EEF0A3F074E6
:10677B0061120DE1126EED120DE1126EC6E8F0A37F
:10678B00E90264A3120DE1126E597406120DE112A7
:10679B006EDEF5838A82E8F0A3E980D27461120D74
:1067AB00E1126EE6E0C0E0741E120DE1D0E0F07471
:1067BB0061120DE1126EED120DE1126EC612643014
:1067CB00741F120DE1A882A9837412120DE1E8F077
:1067DB00A3E9026CD37461120DE1126F05120DE186
:1067EB001264307406120DE1126F05120DE1E024F4
:1067FB0002FAA3E03400FB7461120DE1126F0B740B
:10680B0002120DE1126430E849700C7402120DE1B2
:10681B007486F0A3740BF0126E0850047E107F2761
:10682B007408120DE1E4F0A380087408120DE11254
:10683B006E12F07402120DE1126E5988828983A3D5
:10684B00AA82AB837402120DE1126F1388828983C3
:10685B00E0600A7408120DE1126E6240CD740212F0
:10686B000DE1126E297412120DE1126430740812CC
:10687B000DE1126EA1F97412120DE1E028F8A3E0FC
:10688B0039F974020267D6740D120DE1E06008EE5F
:10689B004F70047E017F007461120DE1126F0512BF
:1068AB000DE1126F59120DE1E0647070387406122D
:1068BB000DE1126EFB120DE1126F34120DE1E024AB
:1068CB0002126EBD120DE1126EC6126430900BB542
:1068DB00120C93741A120DE1120C9F7405120DE138
:1068EB00E4F00269D7EAA2E07406501B120DE11224
:1068FB006E78120C937414120DE1120C9F74061225
:10690B000DE1E024048012120DE1126EFB120DE179
:10691B00126F34120DE1E02402126EBD120DE11262
:10692B006EC6126F59120DE1E0646F7005900BB9D2
:10693B00809EE064757096900BBD80947461120D0F
:10694B00E1126F05120DE1126430EAA2E0740650F9
:10695B0016120DE1126E787808120C757406120D72
:10696B00E1E02404F8801B120DE1126E9BA3E0F50D
:10697B00093395E0F50AF50B7406120DE1E02402DC
:10698B000808126EBE120DE1126F41120DE178086C
:10699B00120C84900B657808120371402174051258
:1069AB000DE1742DF07414120DE17808120C75784A
:1069BB0008120C3E7414120DE17808120C84900B23
:1069CB00BD120C93741A120DE1120C9F744F120D21
:1069DB00E1A882A9837402120DE1126430741212C1
:1069EB000DE1126F44120DE17808120C75E50845A4
:1069FB0009450A450B60097411120DE174018006FB
:106A0B007411120DE1E4F0EE4F7008E0A2E04003C8
:106A1B00026ACB7402120DE1126E72120DE1126F4B
:106A2B0044120DE1780C120C75741A120DE17808F2
:106A3B00120C75780C7908120B6374752508F582A6
:106A4B00740B3509F583E0C0E07402120DE1126E90
:106A5B0078D0E0F07414120DE1780C120C75741AE6
:106A6B00120DE17808120C75780C7908120B63740F
:106A7B0014120DE1780C120C847414120DE17808C9
:106A8B00120C75E5084509450A450B7086126E0810
:106A9B00502E740E120DE1E060267405120DE1E02C
:106AAB006004D2F08002C2F0740A120DE1126E1B68
:106ABB00800E7402120DE1126F25120DE1126E851C
:106ACB007402120DE1126E29744F120DE1C082C0D7
:106ADB00837402120DE1126E49D083D082E582C31A
:106AEB009AFAE5839BFBC3EA9EEB126E6B40C37471
:106AFB000D120DE1E07003026CD47411120DE1E084
:106B0B00A2E04003026CD47404120DE1E0647860DF
:106B1B0005E06458701E1263D3E824FF18E934FFB4
:106B2B00F97402120DE1126F25120DE1126E7874D9
:106B3B0030026CD3E0646F6003026CD47402120DEC
:106B4B00E1126ED964307003026CD480D4740812D5
:106B5B000DE17401F0A3E4F07404120DE1E024FEE6
:106B6B00F0EE4F700F7E018012E4F07408120DE10D
:106B7B00E4F0A3F0126E0850047E067F00746112DD
:106B8B000DE1126F05120DE11264307406120DE166
:106B9B00126E78780C120C757406120DE1E0240459
:106BAB00126EBD120DE1126F41120DE1780C120C39
:106BBB0084900B657808120C75780C7908120575A2
:106BCB0050227405120DE1742DF07414120DE1783E
:106BDB0008120C75E50BB2E7F50B7414120DE17886
:106BEB0008120C84740A120DE1126E59741E120DE8
:106BFB00E1E58228F8E58339F97402120DE112649C
:106C0B0030740D120DE1E0F5087808120EAA740924
:106C1B00120DE1E0F5087808120EAA7404120DE1CA
:106C2B00120EB98E088F097808120EA6740A120D6F
:106C3B00E1E0F9741A120DE1120C93125F3C740629
:106C4B00120DAC7412120DE1126F13740E120DE1D2
:106C5B00E060767405120DE1E06004D2F08002C2B0
:106C6B00F0740A120DE1126E1B7412120DE1C08248
:106C7B00C0837402120DE1126E59D083D082E0C32F
:106C8B0098F8A3E099F9C3E89EE9126E6B503A7439
:106C9B0002120DE1126E72120DE1126F25120DE14F
:106CAB00126E8580C4851082851183126E32126438
:106CBB00297402120DE17495F0A3740BF074121287
:106CCB000DE17498F0A3740BF07412120DE1C082F5
:106CDB00C0837402120DE1126E59D083D082E0C3CF
:106CEB0098FEA3E099FF740A120DE1126E62500A2E
:106CFB007408120DE1E4F0A380307405120DE1E08D
:106D0B006004D2F08002C2F0740A120DE1E0C39E5F
:106D1B00F8A3E09FF9A2F0E433FAE89AF8E99400BB
:106D2B00F97408120DE1E8F0A3E9F0740C120DE10F
:106D3B00E0702B8019745F120DE1126E4F120DE192
:106D4B00126E78120DEB740F120DE1126F6774084F
:106D5B00120DE1126F19120DE112640650D7740572
:106D6B00120DE1E06050745F120DE1126E49740573
:106D7B00120DE1E0F97418120DE1126E78120DEBA1
:106D8B00802C745F120DE1126E497402120DE11228
:106D9B006E92F97418120DE1126E78120DEB7402EB
:106DAB00120DE1126E3B7402120DE1126430740F7E
:106DBB00120DE1126F67EE24FF1EEF34FFFFC312BB
:106DCB006E0A50BE740C120DE1E070030264A474E1
:106DDB0008120DE1126F19120DE112640650030235
:106DEB0064A4745F120DE1126E4F120DE1126E78F6
:106DFB00120DEB740F120DE1126F6780D2C3EF947B
:106E0B0000A2D265D03322E02401F0A3E0340022AB
:106E1B00A2F0E433F8E098FEA3E09400FF22126E98
:106E2B002D22126E32F922E024FFF8A3E034FF2268
:106E3B00E0126E40222401F8A3E03400F922E0FABC
:106E4B00A3E0FB22E0FAA3E0FB7920741822126E78
:106E5B00AE22126EAEE822C3E09EA3E0126E6B224E
:106E6B009FA2D265D03322126E2D740222126E7C39
:106E7B0022E0F8A3E0F583888222126E7C7430F056
:106E8B0022851082851183126E9622126EB4E02237
:106E9B00126E96F50822126EAEC3E498F8E49922AE
:106EAB00126EB4E0F8A3E0F922E0F8A3E0F58388D2
:106EBB008222F8A3E03400F9746122126ECA22E038
:106ECB00FAA3E0F5838A8222851082851183126EE4
:106EDB00CAE022126ECAE0FAA3E022126E96126E7C
:106EEB007D22126E962402F8A3E03400F97461221D
:106EFB00126EABE8FAE9FB741422126EAB74062225
:106F0B00E0FCA3E0F5838C82EAF0A3EBF022E02413
:106F1B00FFF0A3E034FFF0740822E8F0A3E9F0746B
:106F2B000222126451F8A3E022EAF0A3EBF0A3E4EF
:106F3B00F0A3F0740622126ECAE8F0A3E9F0741401
:106F4B0022851082851183E0240108126F7FE8F0FF
:106F5B00A3E9F0740422851082851183E02401F0EB
:106F6B00A3E03400F02212644D2401F8126F7FE885
:106F7B00F0A3E922A3E03400F98510828511832266
:106F8B0000000000000000000000000000000000F6
:106F9B00000000000010000000000000001E0000B8
:106FAB0000000000001FC00000000000001FF800E0
:106FBB0000000000000FFF00000000000001FFE0D8
:106FCB000000000000003FFC00000000000007FC78
:106FDB0000000000000000FC00000000000000FCAE
:106FEB0000000000000003F800000000000007E0B4
:106FFB00000018E801000FC0000018EC00001F8013
:10700B000000181E00007E000000180E8000FC001F
:10701B0000001803C001F80000001801E107F000A0
:10702B0000001800790FC000000018003E1F800000
:10703B00000018000E1FC00000001800031FF8000E
:10704B00000018000F0FFF00000018000D01FFE0FB
:10705B000000180079003FFC00001800F00007FC4E
:10706B0000001801C00000FC000018038000001C89
:10707B0000001807018000000000181C0000000031
:10708B000000181800000000000008B000100000FD
:10709B00000009F0001E0000000019C0001FC00016
:1070AB0000001F01199FF80000001E99001FFF0030
:1070BB000098DC000019FFE00880380000183FE062
:1070CB0008007800011837E00001D800011830E003
:1070DB000001880000183060000B180000183060A9
:1070EB00000E080000183060001C180000183060FB
:1070FB00007808000198306000E01800001830603C
:10710B0001C008000018006007800800001800602C
:10711B000F0018000008006012000800000000605B
:10712B001C0018000180006078000800000000605F
:10713B0070001800000000606000080000100000E4
:10714B003C000800001E00001F000800009FC0004C
:10715B0007800800019FF80001E80800000FFF00FE
:10716B00007808000001FFE0002E080000003FE05F
:10717B00000B8800008007E00001C808898000E050
:10718B0000017C88880000000000FC8800000000E3
:10719B0000489E000010000008801F40001E0000E9
:1071AB00000009D0019FC000000008F4001FF80088
:1071BB0000000C2C001FFF000000080F8019FFE0DF
:1071CB000000080580183FE000000C00C01807E025
:1071DB0000000800F99800E000000C003C180000CB
:1071EB00000008000F18000000000C00071800003A
:1071FB00000008000318000000000C0006980000B7
:10720B0000000C001C98000000000800381800005B
:10721B0000000C006808000000000800E0000000FF
:10722B0000000C03808000000000080700800000B5
:10723B0000000C1C000000000000081800000000FB
:10724B0000000838000E000000000CE0001F0000DA
:10725B00400008C0009F800000000F84881F800042
:10726B0000000EC8001D8F00000C5C00001C1FE00E
:10727B0044845C00001C1FF804C07C00001C1FF839
:10728B0000006C00009C1CFC0001AC00001C1C1CD2
:10729B0000038C00001C1C1C00070C00001C1C1C99
:1072AB00401C0800001C1C1C00180400009C1C1C2B
:1072BB0000680400009C1C1C00E00C00001C1C1C43
:1072CB0001800C00001C1C1C03800C00001E1C1CED
:1072DB0046000400009FDC1C1A000C00008FFC1CF5
:1072EB00180004000007FC1C380004000001FC7CA3
:1072FB0070000C000000387C7B0004000000007C58
:10730B004F000C000080007C05A004000000000072
:10731B0000E80C0000000000003E0400000000002C
:10732B00000F0C00000000004003A4001F9E000093
:10733B000002E42AFF9FC00000007C7FC01FF80002
:10734B000000FFC0001FFF0000BFAE800019FFC090
:10735B007FD00DC000983FE0200005B8001807E073
:10736B000000041A001800E00000040E0018006072
:10737B0000000407C018006000000401C018006082
:10738B004000040078980060000004001C180060A6
:10739B00000004000718006000000400079E006056
:1073AB0000000400019F806040000400038F886090
:1073BB00400004000E878F6000000400080107E006
:1073CB0000000400380007E000000400F00003E0B8
:1073DB0000000402800000C0400004018000000097
:1073EB00000004060000000000000416001E000050
:1073FB000000041C001FC00000000448001FF80020
:10740B00000004E0001FFF00400004C04419FFC04F
:10741B000000078400183FE000002E00001807E072
:10742B0000040C00001800E000041C0000180060B1
:10743B004400340000180060000050000018006089
:10744B000000E400001800600003840000180060D6
:10745B000005040000180060400C040000180060D8
:10746B00001804000018006000780400001E006083
:10747B0000400400001FC06001C00400000FF86052
:10748B00038000000007FF60450004000001FFE0DF
:10749B000C00000000003FE018000400000007E0B3
:1074AB0010000400000000C01800020000000000E3
:1074BB003E0004000000000005A0040000000000D6
:1074CB0000D000000010000000110400001E00009E
:1074DB00000E0000001FC0000005C000001FF800D8
:1074EB000001E400000FFF00000034000001FFE08A
:1074FB0000001E4000007FE000004780000067E0B6
:10750B00002004E0000060E0400000AC0000606080
:10751B000000000E000060600000040320006060AB
:10752B000000040120006060000004016000606046
:10753B00000000003C006060000000000E00606076
:10754B000000000003006060000004000180786010
:10755B000000000001807FE00000000002003FE01F
:10756B000000040006001FE0000000000C0007E014
:10757B0000000400180000C00000040060100000B0
:10758B0000000400A01E000000000401801FC000CA
:10759B0000000407801FF80000000004001FFF001C
:1075AB000000000C0019FFE00000043800183FE059
:1075BB00000004A0001837E0000000E0001830E0E5
:1075CB0000000380001830600000070000183060D6
:1075DB00000006000018306000000C00001830603E
:1075EB000000180000183060000014000018306014
:1075FB000000E0000018006000018400001800602B
:10760B000004000000080060000604000000006099
:10761B000012040000000060001000000000006079
:10762B00002004000000006000600000000000006B
:10763B0000C00000000000000180040000000000FA
:10764B0002000000000000000C0000000000000021
:10765B0008000400000000000C0004000000000003
:10766B000580040000000000014004000000000041
:10767B000030000000000000001D040000000000AE
:10768B00000D4000000000000000D00000000000D2
:10769B000000B0000000000000001400000000001B
:1076AB0000000000000000000000000000100000BF
:1076BB0000000000001C000000000000001E000085
:1076CB0000000000001F000000000000001F000071
:1076DB0000000000001F810000000000001F81E07F
:1076EB0000000000001DC1F800000000001DC1F8E3
:1076FB0000000000001CE0FC003FF01FF81CE01C29
:10770B00003FF01FF81C701C00030001981C701C3C
:10771B0000030001981C381C00030001981C381C46
:10772B0000030001981C1C1C00030001981C1C1C6E
:10773B0000030000181E0E1C00030000181FC61CBF
:10774B0000030000180FC71C003FF0000007C3FC2C
:10775B00003FF000000183FC00000000080001FC6A
:10776B0000000000780000FC00000001F0000008A1
:10777B000000000F800000000000101E0000000041
:10778B000000F01E000000000003E0078000000076
:10779B00001F0000F0100000003C0000381E00002D
:1077AB00003C0000F81E0000000F0003C01E00008C
:1077BB000001E01E001E00000000701C000E000007
:1077CB000001F00F0000000000078001E000000046
:1077DB00003C0000780000000038000008000000AA
:1077EB00001E0000000000000003C00000000000AD
:1077FB000000F0000000000000001000000000007E
:10780B00000000000000000000000000000E00005F
:10781B0000000000001FC00000000000001FF80067
:10782B0000000000001FFF0000000000001DFFE033
:10783B0000000000041C3FF800000000041C07F8C7
:10784B0000000000061C00FC0000001FFE1C001CBA
:10785B000000001FFE1C001C00000000001C001C90
:10786B00001C3800001C001C003C3C00001C001CD1
:10787B0000300C00001C001C00300C00001C001C15
:10788B0000300C00001C001C00318C00001C001C84
:10789B0000318C00001E001C00318C00001FC01C2E
:1078AB0000318C00000FF81C00318C000007FF1C0E
:1078BB00003FFC000001FFFC001F780000003FFCB4
:1078CB0000000000000007FC00000000000000FCAE
:1078DB000000001C000000000000001C0000000065
:1078EB000000001C00000000000000000000000071
:1078FB00003800000000000000380000000000000D
:10790B000038000000000000000000000000000034
:10791B0000000000000000000000000E1C00000032
:10792B000000001E1E0000000000001806000000F2
:10793B0000000018060000000019F01806000000F7
:10794B000030FC18C60000000030CC18C600000048
:10795B000030CC18C60000000030CC18C600000068
:10796B000030CC18C60000000030CC1FFE00000019
:10797B000030CC0FBC0000000030CC000000000039
:10798B000030CC000000000000198C00000000004B
:10799B00001F800000000000000F0000000000002E
:1079AB0000000000000000000000001FFE000000AF
:1079BB000000001FFE000000000000180600000081
:1079CB000000001806000000000000180600000070
:1079DB000000001806000000000000180600000060
:1079EB000000001806000000000000180600000050
:1079FB0000000018060000000000001C0E00000034
:107A0B000000000E1C00000000000007F800000042
:107A1B0000000003F0000000000000000000000068
:107A2B00000000000000000000000000000000004B
:107A3B00000000000000000000000000000000003B
:107A4B00000000000000FF33FF33000000000000C7
:107A5B0000000700070000000000070007000000FF
:107A6B002001FE1FFE1F20012001FE1FFE1F200113
:107A7B0038063C0E6408FF3FFF3F84091C0F1807B4
:107A8B001E30331C1E07C00170001C1E0733011E65
:107A9B001E1FB331E120E120B3311E1F001B8031CB
:107AAB000000000000000B000700000000000000B9
:107ABB0000000000F807FF3F07380000000000003F
:107ACB0000000000000000000000000000000000AB
:107ADB00000000000000000000000000000000009B
:107AEB00000000000000000000000000000000008B
:107AFB00000000000000000000000000000000007B
:107B0B00000000000000000000000000000000006A
:107B1B0000000000000000300030000000000000FA
:107B2B000030003C000FC003F0003C000F000300CE
:107B3B00FC0FFE1F0336812161201B30FE1FFC0F43
:107B4B00042004200620FF3FFF3F002000200020E0
:107B5B000C380E3C032601238121C3207E203C20C0
:107B6B00061803304120412041204120E330BE1F45
:107B7B00000FE00FFC081F08833F803F0008000840
:107B8B003F0C3F1C2130212021206130C11F810F70
:107B9B00E00FF81F5C3046204320C130811F010FDE
:107BAB00010001000100013C813FF1037F000F0048
:107BBB001C0FBE1FE33041204120E330BE1F1C0FC2
:107BCB003C207E20C32081308118830EFE07FC01F0
:107BDB00000000000000000000000000000000009A
:107BEB00000000000000000000000000000000008A
:107BFB00000000000000000000000000000000007A
:107C0B002001200120012001200120012001200161
:107C1B000000000000000000000000000000000059
:107C2B000000000000000000000000000000000049
:107C3B000000000000000000000000000000000039
:107C4B00FC3FFE3F0301010101010301FE3FFC3F2D
:107C5B00FF3FFF3F412041204120E330BE1F1C0F5F
:107C6B00FC0FFE1F03300120012003300E1C0C0CF7
:107C7B00FF3FFF3F0120012001200738FE1FF807BF
:107C8B00FF3FFF3F41204120412041204120012067
:107C9B00FF3FFF3F810081008100810081000100D7
:107CAB00FC0FFE1F03300120812083308E1F8C0FB1
:107CBB00FF3FFF3F4000400040004000FF3FFF3FC1
:107CCB00012001200120FF3FFF3F01200120012067
:107CDB00000C001C0030002000200030FF1FFF0FA5
:107CEB00FF3FFF3FC000E00138071C0E0F3C033085
:107CFB00FF3FFF3F0020002000200020002000203D
:107D0B00FF3FFF3F7800C003C0037800FF3FFF3FFA
:107D1B00FF3FFF3F1C007000C0010007FF3FFF3F0C
:107D2B00FC0FFE1F0330012001200330FE1FFC0F50
:107D3B00FF3FFF3F810081008100C3007E003C00BC
:107D4B000000000000000000000000000000000028
:107D5B00FF3FFF3F810081008101C31F7E3E3C201E
:107D6B003C0C7E1C6330E120C12183318E1F0C0F34
:107D7B00030003000300FF3FFF3F0300030003006A
:107D8B00FF0FFF1F0030002000200030FF1FFF0FF0
:107D9B003F00FF01C00F003C003CC00FFF013F0044
:107DAB00FF01FF3F003EC001C001003EFF3FFF014E
:107DBB0000000000000000000000000000000000B8
:107DCB0000000000000000000000000000000000A8
:107DDB000138013E8127C121612039201F20072056
:107DEB000000000000000000000000000000000088
:107DFB000000000000000000000000000000000078
:107E0B000000000000000000000000000000000067
:107E1B000000000000000000000000000000000057
:107E2B000000000000000000000000000000000047
:107E3B000000000000000000000000000000000037
:107E4B00001E403F2021202120212011E03FC03F78
:107E5B00FF3FFF3F4010202020206030C01F800FCD
:107E6B00800FC01F60302020202020206030401069
:107E7B00800FC01F6030202020204010FF3FFF3FAD
:107E8B00800FC01F6032202220226022C03380135B
:107E9B0020002000FE3FFF3F2100210023000200B5
:107EAB008007C00F6018201020104008E03FE03F13
:107EBB00FF3FFF3F4000200020006000C03F803F9D
:107ECB00000020202020E33FE33F002000200000A3
:107EDB000000000000000000000000000000000097
:107EEB00FC3FFC3F00060007800DC01860302020CF
:107EFB00000001200120FF3FFF3F00200020000079
:107F0B00E03FE03F6000C01FC01F6000E03FC03F8C
:107F1B00E03FE03F4000200020006000C03F803F7A
:107F2B00800FC01F6030202020206030C01F800FCA
:107F3B00E03FE03F400420082008600CC0078003AE
:107F4B000000000000000000000000000000000026
:107F5B00E03FE03FC0004000600060006000400078
:107F6B00C010E0312021202320262024603C401823
:107F7B00000020002000FE1FFE3F202020200000DC
:107F8B00E01FE03F0020002000200010E03FE03F1A
:107F9B00F003F007001C00300030001CF007F0036A
:107FAB00E007E03F0038C007C0070038E03FE007BC
:107FBB006030E03D800D00070007800DE03D603034
:107FCB00E001E027002600380018000EE007E00172
:107FDB0020302038202C20262023A021E0206020D8
:107FEB0018000C000600FF3FFF3F06000C001800B6
:107FFB00000000000000FF3FFF3F000000000000FA
:10800B000006000C0018FF3FFF3F0018000C000695
:10801B000000000000000000000000000000000055
:10802B000000000000000000000000000000000045
:10803B0001F800F860F880F8C0F8E0F820F940F992
:10804B0080F9A0F9E0F900FA40FA60FAA0FAC0FA58
:10805B0000FB20FB60FB80FBC0FBE0FB20FC40FC3B
:10806B0080FCA0FCE0FC00FD40FD60FDA0FDC0FD20
:10807B0000FE20FE60FE80FEC0FEE0FE20FF40FF03
:10808B0080FFA0FFE0FFE0FFE0FFE0F7E0EFE0E7BD
:10809B00E0E7E0DFE0D7E0CFE0CFE0C7E0BFE0B75D
:1080AB00E0B7E0AFE0A7E09FE09FE097E08FE087CD
:1080BB00E087E07FE077E06FE06FE067E05FE0573D
:1080CB00E057E04FE047E03FE03FE037E02FE027AD
:1080DB00E027E01FE017E00FE00FE007E007E00705
:1080EB00E107E207E307E307E407E507E607E6072F
:1080FB00E707E807E907E907EA07EB07EC07EC07EF
:10810B00ED07EE07EF07EF07F007F107F207F207AE
:10811B00F307F407F507F507F607F707F807F8076E
:10812B00F907FA07FB07FB07FC07FD07FE07FE072E
:10813B00FF07FF07DF079F077F073F071F07DF06C5
:10814B00BF067F065F061F06FF05BF059F055F0580
:10815B003F05FF04DF049F047F043F041F04DF037C
:10816B00BF037F035F031F03FF02BF029F025F0278
:10817B003F02FF01DF019F017F013F011F01DF0074
:10818B00BF007F005F001F001F001F001F081F1094
:10819B001F181F181F201F281F301F301F381F408C
:1081AB001F481F481F501F581F601F601F681F70FC
:1081BB001F781F781F801F881F901F901F981FA06C
:1081CB001FA81FA81FB01FB81FC01FC01FC81FD0DC
:1081DB001FD81FD81FE01FE81FF01FF01FF81FF854
:1081EB001FF81EF81DF81CF81CF81BF81AF819F8E4
:1081FB0019F818F817F816F816F815F814F813F804
:10820B0013F812F811F810F810F80FF80EF80DF823
:10821B000DF80CF80BF80AF80AF809F808F807F843
:10822B0007F806F805F804F800000000000000004D
:10823B0000000000000000002000200020002000B3
:10824B00410841084108410861086108610861085B
:10825B008210821082108210A210A210A210A21003
:10826B00C318C318C318C318E318E318E318E318AB
:10827B00042104210421042124212421242124214B
:10828B0045294529452945296529652965296529F3
:10829B008631863186318631A631A631A631A6319B
:1082AB00C739C739C739C739E739E739E739E73943
:1082BB0008420842084208422842284228422842E3
:1082CB00494A494A494A494A694A694A694A694A8B
:1082DB008A528A528A528A52AA52AA52AA52AA5233
:1082EB00CB5ACB5ACB5ACB5AEB5AEB5AEB5AEB5ADB
:1082FB000C630C630C630C632C632C632C632C637B
:10830B004D6B4D6B4D6B4D6B6D6B6D6B6D6B6D6B22
:10831B008E738E738E738E73AE73AE73AE73AE73CA
:10832B00CF7BCF7BCF7BCF7BEF7BEF7BEF7BEF7B72
:10833B001084108410841084308430843084308412
:10834B00518C518C518C518C718C718C718C718CBA
:10835B009294929492949294B294B294B294B29462
:10836B00D39CD39CD39CD39CF39CF39CF39CF39C0A
:10837B0014A514A514A514A534A534A534A534A5AA
:10838B0055AD55AD55AD55AD75AD75AD75AD75AD52
:10839B0096B596B596B596B5B6B5B6B5B6B5B6B5FA
:1083AB00D7BDD7BDD7BDD7BDF7BDF7BDF7BDF7BDA2
:1083BB0018C618C618C618C638C638C638C638C642
:1083CB0059CE59CE59CE59CE79CE79CE79CE79CEEA
:1083DB009AD69AD69AD69AD6BAD6BAD6BAD6BAD692
:1083EB00DBDEDBDEDBDEDBDEFBDEFBDEFBDEFBDE3A
:1083FB001CE71CE71CE71CE73CE73CE73CE73CE7DA
:10840B005DEF5DEF5DEF5DEF7DEF7DEF7DEF7DEF81
:10841B009EF79EF79EF79EF7BEF7BEF7BEF7BEF729
:10842B00DFFFDFFFDFFFDFFFFFFFFFFFFFFFFFFFD1
:10843B000000000000000000000000000000000031
:10844B000000000000000000000000000000000021
:10845B00000102030405060708090A0B0C0D0E0F99
:10846B00101112131415161718191A1B1C1D1E1F89
:10847B00202122232425262728292A2B2C2D2E2F79
:10848B00303132333435363738393A3B3C3D3E3F69
:10849B00404142434445464748494A4B4C4D4E4F59
:1084AB00505152535455565758595A5B5C5D5E5F49
:1084BB0000000000000000000000000000000000B1
:1084CB0000000000000000000000000000000000A1
:1084DB000000000000000000000000000000000091
:1084EB000000000000000000000000000000000081
:1084FB000000000000000000000000000000000071
:10850B000000000000000000000000000000000060
:10851B000000000000000000000000000000000050
:10852B000000000000000000000000000000000040
:10853B000040206010503070084828681858387870
:10854B0004442464145434740C4C2C6C1C5C3C7C20
:10855B0002422262125232720A4A2A6A1A5A3A7A30
:10856B0006462666165636760E4E2E6E1E5E3E7EE0
:10857B000141216111513171094929691959397920
:10858B0005452565155535750D4D2D6D1D5D3D7DD0
:10859B0003432363135333730B4B2B6B1B5B3B7BE0
:1085AB0007472767175737770F4F2F6F1F5F3F7F90
:1085BB0000402060105030700848286818583878F0
:1085CB0004442464145434740C4C2C6C1C5C3C7CA0
:1085DB0002422262125232720A4A2A6A1A5A3A7AB0
:1085EB0006462666165636760E4E2E6E1E5E3E7E60
:1085FB0001412161115131710949296919593979A0
:10860B0005452565155535750D4D2D6D1D5D3D7D4F
:10861B0003432363135333730B4B2B6B1B5B3B7B5F
:10862B0007472767175737770F4F2F6F1F5F3F7F0F
:10863B00008040C020A060E0109050D030B070F0AF
:10864B00088848C828A868E8189858D838B878F81F
:10865B00048444C424A464E4149454D434B474F44F
:10866B000C8C4CCC2CAC6CEC1C9C5CDC3CBC7CFCBF
:10867B00028242C222A262E2129252D232B272F24F
:10868B000A8A4ACA2AAA6AEA1A9A5ADA3ABA7AFABF
:10869B00068646C626A666E6169656D636B676F6EF
:1086AB000E8E4ECE2EAE6EEE1E9E5EDE3EBE7EFE5F
:1086BB00018141C121A161E1119151D131B171F11F
:1086CB00098949C929A969E9199959D939B979F98F
:1086DB00058545C525A565E5159555D535B575F5BF
:1086EB000D8D4DCD2DAD6DED1D9D5DDD3DBD7DFD2F
:1086FB00038343C323A363E3139353D333B373F3BF
:10870B000B8B4BCB2BAB6BEB1B9B5BDB3BBB7BFB2E
:10871B00078747C727A767E7179757D737B777F75E
:10872B000F8F4FCF2FAF6FEF1F9F5FDF3FBF7FFFCE
:10873B003235306E733F3530306E733F312E3075BE
:10874B00733F312E3575733F322E3075733F322E9A
:10875B003575733F35202075733F372E3575733F55
:10876B0031302075733F32302075733F32352075B1
:10877B00733F33302075733F33352075733F34307F
:10878B002075733F34352075733F35302075733F3B
:10879B0036302075733F37302075733F3735207572
:1087AB00733F38302075733F39302075733F31304C
:1087BB003075733F31353075733F32303075733FE1
:1087CB0032353075733F35303075733F312E306D28
:1087DB00733F322E306D733F3530306E733F312E19
:1087EB003075733F322E3075733F332E3075733FB8
:1087FB00342E3075733F352E3075733F3130207505
:10880B00733F31352075733F32302075733F3430F1
:10881B002075733F35302075733F36302075733FAD
:10882B0037302075733F38302075733F39302075E2
:10883B00733F31303075733F31323075733F3134A4
:10884B003075733F31353075733F31363075733F4B
:10885B0031383075733F32303075733F333030758C
:10886B00733F34303075733F35303075733F312E75
:10887B00306D733F322E306D733F342E306D733F3E
:10888B00C082C0838A828B83128920E9F08A828B13
:10889B0083E02401FCA3E03400FD8A828B83ECF09F
:1088AB00A3EDF0D083D0822274F7120E0074FC1269
:1088BB000D967402120DE1EAF0A3EBF0ECFAEDFB6E
:1088CB00740D120DE1A882A983851082851183E8AE
:1088DB00F0A3E9F0851082851183858208858309D1
:1088EB007808120EA67404120DE18582088583099F
:1088FB007808120EA67C8B7D8812645A7404120DB4
:10890B00AC7402120DE1128920E4F07404120DAC68
:10891B007F02020E66E0F8A3E0F583888222FFFF58
:10892B000000020004000600080012001C002600D4
:10893B004E00620076008A009E00B200C600EE0078
:10894B0016012A013E0166018E0156021E03E60343
:10895B000200040008003235306D3F3530306D3F7A
:10896B00312E32353F322E35303F352E30303F31C0
:10897B00322E353F32352E303F35302E303F3132AF
:10898B00356D3F3235306D3F3632356D3F312E32DE
:10899B00353F322E35303F362E32353F31322E3584
:1089AB003F32352E303F0C000B000A000900080047
:0689BB000A00090008009B
:04000005000000B245
:00000001FF
